:0200000480007A
:10000000B72F0000938F0F8073900F3015A8130047
:100010000000130000001300000013000000130094
:100020000000130000001300000013000000130084
:100030000000130000001300000013000000010086
:10004000970200009382020C73905230814001416C
:100050008141014281420143814301448144014580
:100060008145014681460147814701488148014950
:100070008149014A814A014B814B014C814C014D20
:10008000814D014E814E014F814F971102009381A6
:1000900021C2170502001305E542979503009385D9
:1000A000257401461122170502001305A53F970587
:1000B00002009385A53F0146C52817A50300130537
:1000C000657297B503009385A57137B6ABAB130680
:1000D000B6BAD92817B103001301C170EF40807D73
:1000E000860293D21200F512638802008242110147
:1000F0006F00001073002030824211017300203025
:10010000711116C0F3222034E3CC02FC82421101AB
:10011000130141F806C20AC40EC612C816CA1ACC88
:100120001ECE22D026D22AD42ED632D836DA3ADCC7
:100130003EDEC2C0C6C2CAC4CEC6D2C8D6CADACC97
:10014000DECEE2D0E6D2EAD4EED6F2D8F6DAFADCA7
:10015000FEDE73252034F32510340A8601A07310C7
:10016000153492402241B2414242D2426243F243AC
:10017000025492542255B2554256D2566257F25703
:10018000064896482649B649464AD64A664BF64B33
:10019000065C965C265DB65D465ED65E665FF65F83
:1001A0001301C1077300203010C16374B50011053D
:1001B000E5BF828000000000000000000000000099
:1001C000000000000000000000000000000000002F
:1001D000000000000000000000000000000000001F
:1001E000000000000000000000000000000000000F
:1001F000197106C00AC20EC412C616C81ACA1ECC8D
:1002000022CE26D02AD22ED432D636D83ADA3EDCC6
:1002100042DEC6C0CAC2CEC4D2C6D6C8DACADECC96
:10022000E2CEE6D0EAD2EED4F2D6F6D8FADAFEDCA6
:100230009702020083A2022723A02200F322103497
:1002400096DEEF006030170102000321A125024174
:10025000F65273901234B72200009382028873A082
:10026000023082403242C2425243E24372448254DC
:100270001255A2553256C2565257E2577258864806
:100280001649A649364AC64A564BE64B764C865C1A
:10029000165DA65D365EC65E565FE65F0961730059
:1002A0002030970202009382E22123A0120023A2B1
:1002B000220023A4320023A6420023A8520023AA2E
:1002C000620023AC720023AE820023A0920223A21C
:1002D000A20223A4B20223A6C20223A8D20223AA06
:1002E000E20223ACF20223AE020323A0120523A2F2
:1002F000220523A4320523A6420523A8520523AADA
:10030000620523AC720523AE820523A0920723A2C7
:10031000A20723A4B20723A6C20723A8D20723AAB1
:10032000E20723ACF207EF40804D170102000321E2
:1003300061170241F65273901234B7220000938283
:10034000028873A0023082403242C2425243E243EA
:10035000724482541255A2553256C2565257E25731
:10036000725886481649A649364AC64A564BE64B45
:10037000764C865C165DA65D365EC65E565FE65FB1
:10038000096173002030970202009382A21383A0B8
:10039000020003A1420083A1820003A2C20083A243
:1003A000020103A3420183A3820103A4C20183A427
:1003B000020203A5420283A5820203A6C20283A60B
:1003C000020303A7420383A7820303A8C20383A8EF
:1003D000020403A9420483A9820403AAC20483AAD3
:1003E000020503AB420583AB820503ACC20583ACB7
:1003F000020603AD420683AD820603AEC20683AE9B
:10040000020703AFC20983AF820782807370043092
:10041000197106C00AC20EC412C616C81ACA1ECC6A
:1004200022CE26D02AD22ED432D636D83ADA3EDCA4
:1004300042DEC6C0CAC2CEC4D2C6D6C8DACADECC74
:10044000E2CEE6D0EAD2EED4F2D6F6D8FADAFEDC84
:100450009702020083A2020523A0220086DEEF108D
:10046000B040170102000321E1030241F6527390EC
:100470001234B72200009382028873A002308240B7
:100480003242C2425243E243724482541255A25550
:100490003256C2565257E257725886481649A649F4
:1004A000364AC64A564BE64B764C865C165DA65DD0
:1004B000365EC65E565FE65F0961730020309707BF
:1004C00002009387E7FE9843FD576305F7007370BA
:1004D000043001A07370043001A041112AC6B24754
:1004E000739047300100410182804111F327403071
:1004F0003EC673F04330B2473E85410182804111D0
:100500002AC62EC432C2B247F1173EC62247B247AE
:1005100098C3B247938787FA3EC61247B24798C33B
:10052000B247A1173EC68E873E87B24798C3B247EF
:10053000D1173EC6170700001307A7F8B24798C3A4
:10054000B2473E8541018280411106C6EF40A0239B
:10055000EF10D014AA8799C3EF1010310100B240F8
:100560004101828041112AC6B24713878700B247F2
:10057000D8C3B2477D5798C7B24713878700B247A1
:10058000D8C7B24713878700B24798CBB24723A09A
:10059000070001004101828041112AC6B24723A809
:1005A000070001004101828001112AC62EC4B24712
:1005B000DC433ECEA2477247D8C3F2479847A247D2
:1005C00098C7F2479C472247D8C3F247224798C7AB
:1005D000A247324798CBB2479C4313871700B247D4
:1005E00098C301000561828001112AC62EC4A2476A
:1005F0009C433ECC6247FD576316F700B2479C4BC5
:100600003ECE31A8B247A1073ECE21A0F247DC433F
:100610003ECEF247DC439C436247E379F7FEF24764
:10062000D843A247D8C3A247DC43224798C7A24772
:10063000724798C7F2472247D8C3A247324798CBA0
:10064000B2479C4313871700B24798C30100056166
:10065000828001112AC6B2479C4B3ECEB247DC4392
:100660003247184798C7B2479C4732475843D8C3C8
:10067000F247DC4332476316F700B2479847F24728
:10068000D8C3B24723A80700F2479C431387F7FF5C
:10069000F24798C3F2479C433E8505618280797199
:1006A00006D622D42AC62EC4B2473ECEF24781E7F0
:1006B0007370043001A0EF202057F2478043F247C7
:1006C000D85FF247BC43BE853A85EF606060AA8779
:1006D0003307F400F247D8C3F24723AC0702F247CE
:1006E0009843F24798C7F2478043F247DC5F13878D
:1006F000F7FFF247BC43BE853A85EF60605DAA878D
:100700003307F400F247D8C7F2477D57F8C3F247E2
:100710007D57B8C7A24799EFF2479C4B8DC7F24768
:10072000C1073E85EF1090402A878547631DF7007B
:10073000F13911A8F247C1073E852D35F24793875D
:1007400047023E850535EF20005185473E85B25072
:10075000225445618280797106D62AC62EC4B2879A
:10076000A303F10002CCB24781E77370043001A00B
:10077000A24799E302CE01A8A2453245EF60405559
:10078000AA8785073ECEF247938747053E85EF301F
:10079000805C2ACAD24785CFA24789E7D247524711
:1007A00098C331A0D24713874705D24798C3D24791
:1007B0003247D8DFD2472247B8C385455245C535B1
:1007C000D247034771002388E704D2473ECCE24773
:1007D00081E77370043001A0E2473E85B250456165
:1007E0008280797106D6AA87A307F1001305400518
:1007F000EF3060562ACEF247B9CFF24723A2070066
:10080000F24723A00700F24723A40700F24723A6DC
:100810000700F24723AC0702F2470547D8DFF2474B
:1008200023A00704F2477D57F8C3F2477D57B8C7A6
:10083000F2470347F1002388E704F247C1073E85EA
:100840001533F247938747023E85293B814601468F
:10085000814572453122F2473E85B2504561828022
:10086000797106D622D42AC6B2473ECCE24781E748
:100870007370043001A0E247C043EF20001DAA8737
:100880006313F402E247DC471387F7FFE247D8C758
:10089000E247DC4791E78146014681456245C92030
:1008A00085473ECE11A002CEF2473E85B25022547B
:1008B00045618280797106D622D42AC62EC4B247F9
:1008C0003ECCE24781E77370043001A0E247C043A9
:1008D000EF20A017AA87631BF400E247DC471387C9
:1008E0001700E247D8C785473ECE0DA08146224675
:1008F00081456245252E2ACE724785476318F70049
:10090000E247DC4713871700E247D8C7F2473E8526
:10091000B250225445618280797106D62AC62EC40F
:10092000B24781E77370043001A02247B24763F5F4
:10093000E7007370043001A0094681453245213D2E
:100940002ACEF24781C7F247224798DFF24781E774
:100950007370043001A0F2473E85B2504561828039
:10096000397106DE2AC62EC432C236C002D6B2475C
:100970003ED4A25781E77370043001A0A24781E7FB
:10098000A257BC4399E3854711A0814781E7737063
:10099000043001A0024789476317F700A257D85FC8
:1009A00085476314F700854711A0814781E773707D
:1009B000043001A0EF20C00AAA8799E3924799E387
:1009C000854711A0814781E77370043001A0EF20B3
:1009D000A025A257985FA257DC5F6366F700024725
:1009E0008947631DF7020246A245225565232AD294
:1009F000A257DC5389CFA257938747023E85EF1059
:100A0000F0122A8785476317F700093421A092570F
:100A100091C3ED3AEF202024854771A8924789E7DA
:100A2000EF206023814741A8B25799E77C083E85B3
:100A3000EF10702785473ED6EF20E021EF10401AD7
:100A4000EF20801EA257F843FD576315F700A25709
:100A500023A20704A257B847FD576315F700A25712
:100A600023A40704EF20201F58007C08BA853E8588
:100A7000EF107026AA879DEB2255EF006071AA87C0
:100A80008DC3A257C1071247BA853E85EF10E070AB
:100A900022551525EF108016AA87E39A07F2BD327A
:100AA0003DB72255092DEF10601515B722552125A8
:100AB000EF10C01481473E85F25021618280797128
:100AC00006D62AC62EC432C236C0B2473ECCE24752
:100AD00081E77370043001A0A24781E7E247BC437D
:100AE00099E3854711A0814781E77370043001A025
:100AF000024789476317F700E247D85F85476314C9
:100B0000F700854711A0814781E77370043001A089
:100B1000E93AAA873ECAE247985FE247DC5F63662C
:100B2000F700024789476315F7040246A24562456C
:100B30009521E247B847FD576313F702E247DC53BC
:100B40008DC7E247938747023E85EF10207EAA8734
:100B500089CF924799CB9247054798C339A0E2477E
:100B6000BC4713871700E247B8C785473ECE11A0A0
:100B700002CED2473E859532F2473E85B25045615E
:100B80008280797106D62AC62EC4B2473ECCE2478F
:100B900081E77370043001A0E247BC4381C77370E2
:100BA000043001A0E2479C4381E7E247DC4399E33C
:100BB000854711A0814781E77370043001A0353269
:100BC000AA873ECAE247985FE247DC5F6377F70493
:100BD000E2479C5F13871700E24798DFE247B84778
:100BE000FD576313F702E247DC538DC7E247938753
:100BF00047023E85EF108073AA8789CFA24799CB21
:100C0000A247054798C339A0E247BC47138717009E
:100C1000E247B8C785473ECE11A002CED2473E85F7
:100C20006D38F2473E85B25045618280397106DEEB
:100C30002AC62EC432C236C002D6B2473ED4A2570C
:100C400081E77370043001A0A24781E7A257BC433B
:100C500099E3854711A0814781E77370043001A0B3
:100C6000EF101060AA8799E3924799E3854711A096
:100C7000814781E77370043001A0EF10F07AA2572A
:100C80009C5FB5CBA257DC473ED2A2452255F92E38
:100C9000824795EFA2579C5F1387F7FFA25798DF13
:100CA000A2579C4391E7EF2060022A87A257D8C33E
:100CB000A2579C4B8DCFA257C1073E85EF1000670E
:100CC0002A8785476315F702EFF04FF40DA0A2576E
:100CD0001257D8C7A257DC5399CBA2579387470224
:100CE0003E85EF10A064AA8799C3EFF02FF2EF10B2
:100CF000907685475DA8924789E7EF10D0758147C8
:100D00006DA0B25799E77C083E85EF10C079854702
:100D10003ED6EF105074EF00B06CEF10F070A25799
:100D2000F843FD576315F700A25723A20704A25703
:100D3000B847FD576315F700A25723A40704EF1027
:100D4000907158007C08BA853E85EF10C078AA875C
:100D5000A1EB2255CD2EAA879DCFA2579C4391EBA4
:100D6000EF10906CA257DC433E85EF107052EF10ED
:100D7000906EA257938747021247BA853E85EF10BF
:100D8000C04122550D2EEF007067AA87E39707EE4A
:100D9000EFF0CFE7DDB52255392EEF003066F1BD1B
:100DA0002255112EEF00906581473E85F25021615A
:100DB0008280797106D62AC62EC432C2B2473ECC92
:100DC000E24781E77370043001A0A24781E7E24760
:100DD000BC4399E3854711A0814781E773700430D4
:100DE00001A0EFF08FF0AA873ECAE2479C5FA1CB3B
:100DF000A2456245A52CE2479C5F1387F7FFE247B7
:100E000098DFE247F843FD576312F702E2479C4B35
:100E100085C7E247C1073E85EF104051AA8789CFB9
:100E2000924799CB9247054798C339A0E247FC43C4
:100E300013871700E247F8C385473ECE11A002CEC4
:100E4000D2473E85EFF06FE9F2473E85B2504561EB
:100E50008280797106D62AC62EC4B2473ECCE247BC
:100E600081E77370043001A0A24781E7E247BC43E9
:100E700099E3854711A0814781E77370043001A091
:100E8000E247BC4381E77370043001A0EFF0EFE567
:100E9000AA873ECAE2479C5F89CFE247DC473EC84B
:100EA000A2456245E122E2474247D8C785473ECE88
:100EB00011A002CED2473E85EFF02FE2F2473E85E9
:100EC000B25045618280797106D62AC6B24781E761
:100ED0007370043001A0EF103055B2479C5F3ECED6
:100EE000EF107057F2473E85B250456182807971AC
:100EF00006D62AC6B2473ECEF24781E77370043069
:100F000001A0EF107052F247D85FF2479C5FB30721
:100F1000F7403ECCEF103054E2473E85B250456179
:100F2000828001112AC6B24781E77370043001A0A4
:100F3000B2479C5F3ECEF2473E8505618280797163
:100F400006D62AC6B2473ECEF24781E77370043018
:100F500001A07245E5247245EF20F0720100B25005
:100F60004561828041112AC6B247FC473E85410156
:100F7000828041112AC62EC4B2472247F8C7010019
:100F80004101828041112AC6B24783C707053E85C9
:100F900041018280797106D62AC62EC432C202CEA1
:100FA000B247BC4391EFB2479C43D5E7B247DC431D
:100FB0003E85EF10903B2ACEB24723A2070061A8DE
:100FC000924785EFB2479847B247BC433E86A24559
:100FD0003A85EF20F079B2479847B247BC433E9735
:100FE000B24798C7B2479847B247DC436365F706F4
:100FF000B2479843B24798C7B9A8B247D847B24753
:10100000BC433E86A2453A85EF209076B247D8474A
:10101000B247BC43B307F0403E97B247D8C7B24788
:10102000D847B2479C43637BF700B247D843B247E7
:10103000BC43B307F0403E97B247D8C71247894731
:10104000631BF700B2479C5F99C7B2479C5F138749
:10105000F7FFB24798DFB2479C5F13871700B2478C
:1010600098DFF2473E85B25045618280011106CE7D
:101070002AC62EC4B247BC439DCBB247D847B2471D
:10108000BC433E97B247D8C7B247D847B247DC43C4
:101090006366F700B2479843B247D8C7B247D8470C
:1010A000B247BC433E86BA852245EF20706C0100F2
:1010B000F24005618280011106CE2AC6EF10D036BB
:1010C00025A0B247DC5395C7B247938747023E85B8
:1010D000EF10C025AA8799C3EF104049B247BC471B
:1010E0001387F7FFB247B8C7B247BC47E34BF0FCE2
:1010F00011A00100B2477D57B8C7EF10D035EF10EF
:10110000B0321DA0B2479C4B8DC7B247C1073E8588
:10111000EF10C021AA8799C3EF104045B247FC43A6
:101120001387F7FFB247F8C3B247FC43E34CF0FC28
:1011300011A00100B2477D57F8C3EF10D031010074
:10114000F24005618280797106D62AC6EF10D02D53
:10115000B2479C5F81E785473ECE11A002CEEF10DB
:10116000902FF2473E85B2504561828001112AC618
:10117000B24781E77370043001A0B2479C5F81E7FA
:1011800085473ECE11A002CEF2473E8505618280A2
:10119000797106D62AC6EF103029B247985FB24758
:1011A000DC5F6315F70085473ECE11A002CEEF103D
:1011B000902AF2473E85B2504561828001112AC6CD
:1011C000B24781E77370043001A0B247985FB2471D
:1011D000DC5F6315F70085473ECE11A002CEF247D3
:1011E0003E850561828001112AC62EC402CE81A0EF
:1011F000178703001307075BF2478E07BA979C43D4
:1012000085E7178703001307E759F2478E07BA9758
:10121000224798C3178703001307C758F2478E0762
:10122000BA973247D8C301A8F24785073ECE724726
:101230009D47E3FFE7FA01000561828001112AC69C
:1012400002CE0DA8178703001307C755F2478E0774
:10125000BA97DC433247631CF70017870300130774
:101260006754F2478E07BA9723A0070001A8F247F8
:1012700085073ECE72479D47E3F6E7FC0100056116
:101280008280797106D62AC62EC432C2B2473ECEBB
:10129000EF109019F247F843FD576315F700F24736
:1012A00023A20704F247B847FD576315F700F2473A
:1012B00023A40704EF10301AF2479C5F89EBF24732
:1012C000938747021246A2453E85EF00907E724505
:1012D000DD330100B25045618280397106DE2ACECD
:1012E0002ECC36C83AC63EC442C246C0B287231B83
:1012F000F100F24781E77370043001A03247A5473F
:1013000063F5E7007370043001A0835761019245D3
:101310003E85EF1080512AD4A257638F0712A2573F
:10132000985B83566101B7070040FD17B6978A079F
:10133000BA973ED29257F19B3ED292578D8B81C77E
:101340007370043001A0835761013E8782463246A4
:10135000E2452255EF10E0274246F2451255EFF0E4
:101360000F9A2A87A25798C3A24781C7A24722573C
:1013700098C3EF10700B97F701009387E72F9C43FA
:101380001387170097F701009387072F98C397F7E4
:101390000100938727119C4395E397F701009387FA
:1013A0006710225798C397F701009387E72C98435B
:1013B0008547631AF702EF10C02C35A097F701009C
:1013C0009387472C9C4385E397F701009387870D0C
:1013D0009C43DC5732476368F70097F70100938717
:1013E000670C225798C397F701009387A72A9C435D
:1013F0001387170097F701009387C72998C397F7BA
:101400000100938727299843A257B8C7A257D857F6
:1014100097F701009387C7269C4363F9E700A2571B
:10142000D85797F701009387A72598C3A257D85795
:10143000BA878A07BA978A0717F701001307471078
:101440003E97A2579107BE853A85EFF0EF95854705
:101450003ED6EF10500019A0FD573ED632578547B3
:101460006313F70297F701009387C7219C4381CF4D
:1014700097F70100938707039C43DC57324763F4D7
:10148000E700EFE0BFF8B2573E85F250216182805D
:10149000797106D62AC6EF102079B24799E797F7F7
:1014A0000100938727009C4311A0B2473ECEF2472C
:1014B00091073E85EFF0EF99F2479C5791C7F247AD
:1014C000E1073E85EFF0EF98F2479107BE8517F5EB
:1014D00001001305A517EFF02F8D97F701009387F3
:1014E00027189C431387170097F701009387471726
:1014F00098C397F701009387E7199C431387170058
:1015000097F701009387071998C3EF10C07497F7F6
:101510000100938727179C439DCB97F70100938782
:1015200067F89C437247631EF70097F701009387A3
:10153000E7169C4381C77370043001A0EFE01FEDF4
:1015400039A0EF10606EEF10A04BEF10C0700100DB
:10155000B25045618280797106D62AC62EC402CE69
:10156000B24781E77370043001A0A24781E773702E
:10157000043001A097F70100938747129C4381C76D
:101580007370043001A0A92D97F701009387070F0E
:101590009C433ECCB2479C432247BA973ECAB247CF
:1015A0009C436247637EF700B2479C435247637493
:1015B000F7025247E24763F0E70285473ECE21A893
:1015C000B2479C4352476366F7005247E24763F4D1
:1015D000E70085473ECEB247524798C3F24789CFCE
:1015E00097F70100938707EC9C4391073E85EFF046
:1015F0004F865245EF10001B11252AC8C24799E3B8
:10160000EFE0DFE00100B25045618280797106D6DB
:101610002AC602CEB247A9C397F7010093870708ED
:101620009C4381C77370043001A05D2B97F70100C4
:101630009387C7049C433247BA973ECC97F7010083
:10164000938747E69C4391073E85EFF08F80624584
:10165000EF10401565232ACEF24799E3EFE01FDB38
:101660000100B25045618280797106D62AC6B24720
:101670003ECCE24781E77370043001A097F7010088
:10168000938747E29C4362476314F70002CEBDA0F4
:10169000EF108059E247DC4B3ECAEF10C05B97F772
:1016A00001009387E7F89C435247630AF70097F7D6
:1016B0000100938727F89C4352476315F700894739
:1016C0003ECE2DA8524797F701009387A7F9631BD9
:1016D000F700E2479C5781E78D473ECE05A089473A
:1016E0003ECE29A8524797F70100938727F6631546
:1016F000F70091473ECE19A085473ECEF2473E8582
:10170000B25045618280797106D62AC6EF10C05169
:10171000B24799E797F701009387C7D89C4311A078
:10172000B2473ECEF247DC573ECCEF10C052E24704
:101730003E85B25045618280797106D62AC6EFE0B7
:10174000DFDAAA873ECEB24799E797F70100938781
:1017500067D59C4311A0B2473ECCE247DC573ECA56
:10176000F2473E85EFE07FD7D2473E85B2504561D4
:101770008280797106D62AC62EC402CE2247A5479A
:1017800063F5E7007370043001A02247A54763F4B6
:10179000E700A5473EC4EF102049B24799E797F705
:1017A0000100938727D09C4311A0B2473ECCE2476B
:1017B000BC4B3ECA5247A247630AF70E2247D247A4
:1017C00063F6E70297F701009387C7CD9C43624712
:1017D0006308F70297F701009387C7CC9C43DC5757
:1017E0002247636FF70085473ECE19A897F701009F
:1017F000938747CB9C4362476314F70085473ECEEF
:10180000E247DC573EC8E247B84BE247DC57631576
:10181000F700E2472247D8D7E2472247B8CBE24752
:101820009C4F63C707002947A2471D8FE24798CF07
:10183000E247D44B4247BA878A07BA978A0717F715
:1018400001001307E7CFBA976394F600854711A00C
:101850008147B9C7E24791073E85EFE09FDFE24746
:10186000D85797F701009387A7E19C4363F9E700F6
:10187000E247D85797F70100938787E098C3E2477C
:10188000D857BA878A07BA978A0717F7010013074C
:1018900027CB3E97E2479107BE853A85EFE0DFD040
:1018A000724785476314F700EFE05FB6EF10A03A88
:1018B0000100B25045618280797106D62AC6EF10C8
:1018C000A036B24799E797F701009387A7BD9C43DD
:1018D00011A0B2473ECEF24791073E85EFE07FD799
:1018E000F2479C5791C7F247E1073E85EFE07FD66C
:1018F000F2479107BE8517F501001305A5D6EFE065
:10190000BFCAEF10403597F701009387A7B99C43F2
:1019100072476319F70497F701009387A7D69C4392
:1019200089CF97F70100938767D79C4381C773706E
:10193000043001A0EFE09FAD91A097F701009387DD
:1019400067D2984397F70100938707D39C436319A5
:10195000F70097F701009387E7B423A0070039A8A1
:10196000212729A897F701009387C7D19C4399C7DE
:10197000EF10802BEF10C008EF10E02D0100B250E7
:101980004561828001112AC602CEB2473ECCB247E1
:1019900081E77370043001A0E247D84B97F701004C
:1019A000938747CC6314F700854711A0814795C3FF
:1019B000E247985797F70100938707C8630BF70032
:1019C000E2479C5799E3854711A0814799C3854712
:1019D0003ECEF2473E8505618280797106D62AC6E1
:1019E000B2473ECEB24781E77370043001A0F247A0
:1019F000C9C797F701009387E7AA9C437247630E14
:101A0000F706EF1060227245B53F2A8785476314B9
:101A1000F706F24791073E85EFE0BFC3F247D8577C
:101A200097F701009387C7C59C4363F9E700F24726
:101A3000D85797F701009387A7C498C3F247D857A0
:101A4000BA878A07BA978A0717F70100130747AFC3
:101A50003E97F2479107BE853A85EFE0FFB4F24723
:101A6000D85797F701009387E7A39C43DC5763643B
:101A7000F700EFE0BF99EF10001E0100B250456182
:101A80008280797106D62AC602CEB2473ECCB247D2
:101A900081E77370043001A0EFE03FA5AA873ECA3A
:101AA0006245CD352A8785476314F70897F701000B
:101AB0009387C7BE9C43A5E7E247D85797F7010035
:101AC0009387479E9C43DC576364F70085473ECE6F
:101AD000E24791073E85EFE0DFB7E247D85797F737
:101AE00001009387E7B99C4363F9E700E247D857C1
:101AF00097F701009387C7B898C3E247D857BA87CA
:101B00008A07BA978A0717F70100130767A33E975A
:101B1000E2479107BE853A85EFE01FA911A8E24789
:101B2000E107BE8517F50100130505B1EFE0DFA75A
:101B3000D2473E85EFE07F9AF2473E85B25045613D
:101B40008280011106CE81480148814701478146C4
:101B50001306004097E501009385C54A171500005C
:101B6000130585A5EFF06FF72AC632478547631541
:101B7000F700EF10C06D2AC6324785476319F70298
:101B80007370043097F70100938707B17D5798C3AE
:101B900097F70100938707AF054798C397F70100B0
:101BA0009387C7AD23A00700EFE0AFEF31A0B247A6
:101BB00081E77370043001A00100F240056182806A
:101BC000411106C67370043097F70100938787AB05
:101BD00023A00700EFE02FFB0100B240410182800B
:101BE00097F70100938787AB9C431387170097F7FC
:101BF00001009387A7AA98C301008280011106CE35
:101C000002C697F70100938767A99C4381E7737029
:101C1000043001A0EF10400197F70100938707A857
:101C20009C431387F7FF97F70100938727A798C373
:101C300097F70100938787A69C436390071097F757
:101C40000100938767A39C436389070E59A097F708
:101C500001009387679EDC47DC473EC4A247E1074B
:101C60003E85EFE01F9FA24791073E85EFE07F9EF4
:101C7000A247D85797F70100938787A09C4363F941
:101C8000E700A247D85797F701009387679F98C34B
:101C9000A247D857BA878A07BA978A0717F7010069
:101CA0001307078A3E97A2479107BE853A85EFE062
:101CB000BF8FA247D85797E701009387A77E9C4321
:101CC000DC576368F70097F701009387279C054767
:101CD00098C397F70100938727969C43ADFB97F72E
:101CE00001009387679A9C438DCF35A0452AAA8728
:101CF00099C797F7010093876799054798C397F7A6
:101D00000100938767989C431387F7FF97F70100BB
:101D10009387879798C397F701009387E7969C432B
:101D2000F1F797F701009387679698438547631605
:101D3000F70085473EC6EFE06FEDEF00D071B24788
:101D40003E85F24005618280011106CEEF00D06D24
:101D500097F70100938787929C433EC6EF00B06FD0
:101D6000B2473E85F24005618280011106CEEFE068
:101D7000CFF7AA873EC697F70100938727909C4329
:101D80003EC4B2473E85EFE04FF5A2473E85F240A4
:101D90000561828097F701009387078E9C433E85FB
:101DA0008280797106D62AC62EC432C202CEA947D5
:101DB0003ECC3D3597F701009387078C9C43224723
:101DC0006368F70CE247FD173ECCF24796073247AF
:101DD000B306F7006247BA878A07BA978A0717E7F8
:101DE00001001307E775BA970546BE853685EF00F3
:101DF000902A2A87F247BA973ECEE247E1F7F247A8
:101E0000960732473E9797F70100938767829C4376
:101E10000946BE853A85EF0010282A87F247BA970F
:101E20003ECEF247960732473E9797F701009387D9
:101E300067809C430946BE853A85EF00D0252A87F6
:101E4000F247BA973ECEF24796073247BA97114605
:101E500097E501009385857F3E85EF00D0232A8793
:101E6000F247BA973ECEF24796073247BA970D46E9
:101E700097E501009385057F3E85EF00D0212A87F5
:101E8000F247BA973ECE924781C7924723A00700F8
:101E9000B533F2473E85B25045618280797106D6EE
:101EA00002CE97E701009387677F9C4363950718ED
:101EB00097E701009387877C9C431387170097E778
:101EC00001009387A77B98C397E701009387077B5F
:101ED0009C433ECCE247B9EF97E7010093874775F3
:101EE0009C439C4381C77370043001A097E70100B5
:101EF000938707749C433ECA97E7010093878773D3
:101F0000984397E701009387A77298C397E701006A
:101F100093874772524798C397E7010093874777A3
:101F20009C431387170097E701009387677698C350
:101F3000EF00102D97E70100938707769C436247D7
:101F40006365F70C97E701009387876E9C439C437A
:101F500099E3854711A0814781CB97E701009387DB
:101F6000A7737D5798C355A097E701009387476CE7
:101F70009C43DC47DC473EC8C247DC433EC6624761
:101F8000B2476379F70097E701009387E77032471C
:101F900098C3A5A8C24791073E85EFE08FEBC247E3
:101FA0009C5791C7C247E1073E85EFE08FEAC247E1
:101FB000D85797E701009387A76C9C4363F9E70024
:101FC000C247D85797E701009387876B98C3C247EA
:101FD000D857BA878A07BA978A0717E70100130705
:101FE00027563E97C2479107BE853A85EFE0CFDB83
:101FF000C247D85797E701009387C74A9C43DC57ED
:10200000E362F7F485473ECE35BF97E7010093873B
:1020100067499C43D85797E6010093866652BA8772
:102020008A07BA978A07B6979843854763F1E7020C
:1020300085473ECE29A897E701009387E7649C4334
:102040001387170097E701009387076498C397E702
:1020500001009387A7639C4399C385473ECEF2470F
:102060003E85B25045618280011106CE97E701009E
:102070009387C7629C4381CB97E7010093870761F1
:10208000054798C339A297E701009387276023A0EB
:10209000070097E701009387E7409C439C5B3EC69F
:1020A000B7A7A5A59387575A3EC4B2479C4322477A
:1020B0006314F702B24791079C432247631EF7005F
:1020C000B247A1079C4322476318F700B247B10704
:1020D0009C4322476308F70497E701009387873CF6
:1020E000984397E701009387E73B9C439387470317
:1020F000BE853A85EF20F00A35A097E70100938767
:1021000027589C4381E77370043001A097E70100D2
:10211000938707579C431387F7FF97E7010093873F
:10212000275698C397E7010093878755984397E60A
:1021300001009386E640BA878A07BA978A07B6975E
:102140009C43C5DF97E70100938787539843BA877D
:102150008A07BA978A0717E701001307673EBA97FD
:102160003EC29247DC43D8439247D8C39247D843F4
:102170009247A1076317F7009247DC43D843924781
:10218000D8C39247DC43D84797E70100938787314C
:1021900098C30100F24005618280797106D62AC693
:1021A0002EC4B24781E77370043001A097E70100A5
:1021B0009387472F9C43E107BE853245EFE0CFC2AE
:1021C00097E701009387072E9C4391073E85EFE038
:1021D0004FC82247FD576310F70297E70100938726
:1021E000672C9C439107BE8517E5010013058547C1
:1021F000EFE08FBB19A897E70100938727489C431E
:102200002247BA973ECE7245712B0100B25045610C
:102210008280797106D62AC62EC432C2B24781E7BF
:102220007370043001A097E70100938727479C4310
:1022300081E77370043001A097E701009387872638
:102240009C43A24637070080558F98CF97E701003F
:10225000938747259C43E107BE853245EFE0CFB425
:1022600097E70100938707249C4391073E85EFE0A1
:102270004FBE1247FD576310F70297E7010093879F
:1022800067229C439107BE8517E501001305853D34
:10229000EFE08FB119A897E701009387273E9C4391
:1022A0001247BA973ECE7245F5290100B2504561FA
:1022B0008280797106D62AC62EC432C2B24781E71F
:1022C0007370043001A097E701009387A71D9C431A
:1022D000E107BE853245EFE02FAD97E70100938718
:1022E000671C9C4391073E85EFE0AFB612478547D8
:1022F0006310F70297E701009387C71A9C43910781
:10230000BE8517E501001305E535EFE0EFA919A833
:1023100097E70100938787369C432247BA973ECEC2
:10232000724549210100B25045618280797106D61B
:102330002AC6B247DC47DC473ECCE24781E77370F0
:10234000043001A0E247E1073E85EFE08FB097E758
:1023500001009387A7349C43A1EBE24791073E8598
:10236000EFE02FAFE247D85797E701009387473157
:102370009C4363F9E700E247D85797E7010093874A
:10238000273098C3E247D857BA878A07BA978A078F
:1023900017E701001307C71A3E97E2479107BE856A
:1023A0003A85EFE06FA011A8E247E107BE8517E587
:1023B000010013056528EFE02F9FE247D85797E704
:1023C00001009387270E9C43DC5763FBE70085479A
:1023D0003ECE97E701009387672B054798C311A06E
:1023E00002CEF2473E85B25045618280797106D6B1
:1023F0002AC62EC497E701009387472A9C4381E7AA
:102400007370043001A02247B70700805D8FB24788
:1024100098C3B247DC473ECCE24781E77370043093
:1024200001A03245EFE0EFA2E24791073E85EFE0E1
:102430004FA2E247D85797E70100938767249C4350
:1024400063F9E700E247D85797E7010093874723EE
:1024500098C3E247D857BA878A07BA978A0717E717
:1024600001001307E70D3E97E2479107BE853A85C5
:10247000EFE08F93E247D85797E7010093878702F1
:102480009C43DC5763FBE70085473ECE97E701009E
:102490009387C71F054798C311A002CEF2473E8518
:1024A000B2504561828041112AC6B24781E77370FC
:1024B000043001A097E701009387871D9843B24736
:1024C00098C397E701009387671B9843B247D8C327
:1024D000010041018280797106D62AC62EC4B24716
:1024E00081E77370043001A0A24781E77370043064
:1024F00001A01D2F97E70100938747189C433ECC0E
:10250000A2479843FD576314F70002CE91A8B24743
:10251000984397E701009387A7179C43630AF70046
:10252000B247DC4362476365F70085473ECE0DA89E
:10253000B247DC4362471D8FA2479C436370F7029A
:10254000A2479843B247D443E247B387F6403E9749
:10255000A24798C33245813F02CE19A085473ECE9F
:10256000DD2DF2473E85B2504561828097E701003C
:102570009387C711054798C30100828001112AC6BD
:10258000B24799C7B2473ECCE247FC473ECE11A0C6
:1025900002CEF2473E850561828001112AC62EC413
:1025A000B24791C7B2473ECEF2472247F8C7010073
:1025B00005618280011106CE2AC6852297E70100B7
:1025C000938707F898438547E3F9E7FEEFD01FE4C8
:1025D000EDB7397106DE2ACE2ECC32CA36C8BA879C
:1025E0002317F10002D625A06247B257BA9703C756
:1025F0000700F246B257B697238AE7026247B257FE
:10260000BA9783C7070089CBB25785073ED63257A2
:10261000BD47E3FBE7FC11A00100F247A3810704DB
:102620005247A54763F4E700A5473ECAF247524721
:10263000D8D7F2475247B8CBF24723AA0704F2474C
:1026400091073E85EFD05FF5F247E1073E85EFD079
:10265000BFF4F247724798CB2947D2471D8FF24704
:1026600098CFF2477247D8D3F24723A20704F24724
:1026700023AC0704F24723AE07040100F2502161A6
:102680008280011106CE02C60DA03247BA878A07A2
:10269000BA978A0717E70100130787EABA973E85BA
:1026A000EFD05FECB24785073EC63247A547E3FE51
:1026B000E7FC17E50100130525F5EFD0BFEA17E5A4
:1026C00001001305A5F5EFD0FFE917E5010013059B
:1026D000A5F6EFD03FE917E50100130525F7EFD088
:1026E0007FE817E501001305E5F7EFD0BFE797E7AF
:1026F00001009387E7F317E701001307E7F098C39A
:1027000097E70100938707F317E70100130707F125
:1027100098C30100F24005618280011106CE8DA8A8
:10272000EFF00FCC97E70100938747F29C4393B7F4
:10273000170093F7F70F3EC6EFF04FCCB247A9EB67
:10274000E52197E70100938767F0DC47DC473EC44B
:10275000A24791073E85EFD0DFEF97E7010093870F
:10276000A7F19C431387F7FF97E701009387C7F012
:1027700098C397E701009387A7EE9C431387F7FF61
:1027800097E701009387C7ED98C3F1212245912C6B
:1027900097E701009387C7EC9C43D9F30100F2400F
:1027A00005618280011106CE2AC697E70100938752
:1027B00067CF9C433247D8C397E70100938707EC64
:1027C0009C4332476372F70297E70100938787E6DD
:1027D000984397E701009387E7CC9C439107BE8518
:1027E0003A85EFD07FE035A897E70100938747E46B
:1027F000984397E701009387E7CA9C439107BE85FA
:102800003A85EFD07FDE97E701009387E7E89C43A6
:1028100032476378F70097E701009387E7E732478D
:1028200098C30100F24005618280797106D6AA87BB
:102830002EC42317F100A24789EB8357E1008A07D2
:102840003E85EF104051AA8711A0A2473ECCE24737
:1028500085C313050006EF1000502ACEF24789C742
:10286000F247624798DB31A06245EF10C06111A0CA
:1028700002CEF24781CFF247985B8357E1008A0787
:102880003E869305500A3A85EF104075F2473E8523
:10289000B25045618280397106DE22DC2AC62EC420
:1028A00032C202D6A2479C43638D070EA2473ED494
:1028B000A257DC43D843A257D8C3A257D843A25744
:1028C000A1076317F700A257DC43D843A257D8C328
:1028D000A257DC43DC473ED2A2473ED08257DC43BE
:1028E000D8438257D8C38257D8438257A10763176A
:1028F000F7008257DC43D8438257D8C38257DC4362
:10290000DC473ECEB25796073247BA97724798C314
:10291000B25796073247BA97724713074703D8C38F
:10292000B25796073247BA977247384798C7B25797
:1029300096073247BA971247D8C7B2579607324719
:10294000BA977247585798CB12478D47631BF700C9
:10295000F2479C5799C7B25796073247BA9709472B
:10296000D8C7B25796073247BA977247384BD8CB79
:10297000B25796073247BA9723AC0700F247945BE9
:10298000B257960732473304F70036850D20AA87E1
:10299000231EF400B25785073ED672479257E31DB7
:1029A000F7F2B2573E85F2506254216182800111E4
:1029B0002AC602CE39A0B24785073EC6F247850730
:1029C0003ECEB24703C707009307500AE305F7FE60
:1029D000F24789833ECEF247C207C1833E85056137
:1029E0008280011106CE2AC6B2479C5B3E85EF105D
:1029F00080493245EF1020490100F2400561828094
:102A0000411197E701009387A7C29C439C4399E338
:102A1000854711A0814781CB97E701009387C7C7FE
:102A20007D5798C305A097E70100938767C09C4333
:102A3000DC47DC473EC6B247D84397E7010093879F
:102A4000A7C598C3010041018280411197E70100A9
:102A5000938747A59C433EC6B2473E85410182808D
:102A6000411197E701009387E7C19C4381E78547C0
:102A70003EC619A897E70100938747C29C4381E7A8
:102A800089473EC611A002C6B2473E8541018280F9
:102A9000797106D62AC6B2473ECEB247F9C3F2478D
:102AA000D85797E701009387E79F9C43DC57637AE9
:102AB000F70AF2479C4F63CC070097E70100938722
:102AC000679E9C43DC5729471D8FF24798CFF247FA
:102AD000D44BF247D857BA878A07BA978A0717E7BD
:102AE00001001307E7A5BA976394F600854711A084
:102AF0008147A5C3F24791073E85EFD09FB597E781
:102B000001009387279A9C43D857F247D8D7F247BA
:102B1000D85797E701009387A7B69C4363F9E7006E
:102B2000F247D85797E70100938787B598C3F247D4
:102B3000D857BA878A07BA978A0717E70100130799
:102B400027A03E97F2479107BE853A85EFD0DFA5D3
:102B500009A897E701009387E7949C43D857F24769
:102B6000D8D70100B25045618280797106D62AC655
:102B7000B2473ECC02CEB247DDC397E70100938750
:102B800067929C4362476305F7007370043001A0AD
:102B9000E247FC4B81E77370043001A0E247FC4B35
:102BA0001387F7FFE247F8CBE247D857E247BC4B21
:102BB0006307F706E247FC4BBDE3E24791073E851A
:102BC000EFD03FA9E247B84BE247D8D7E247DC57FE
:102BD00029471D8FE24798CFE247D85797E7010072
:102BE000938707AA9C4363F9E700E247D85797E722
:102BF00001009387E7A898C3E247D857BA878A07A6
:102C0000BA978A0717E70100130787933E97E247B1
:102C10009107BE853A85EFD03F9985473ECEF24772
:102C20003E85B250456182807370043097E70100A1
:102C3000938747A59C4391CF97E7010093878786A9
:102C40009C43F8430507F8C397E7010093878785FE
:102C50009C430100828097E701009387A7A29C43D1
:102C60008DCB97E701009387E7839C43FC4395C393
:102C700097E70100938707839C43F8437D17F8C3C8
:102C800097E70100938707829C43FC4399E37360B5
:102C9000043001008280411197E70100938787800B
:102CA0009C439C4F3EC697D701009387A77F9C43C8
:102CB000D85797D701009387E77E9C43A94633876F
:102CC000E64098CFB2473E854101828097D7010008
:102CD0009387477D9C4389CB97D701009387877C57
:102CE0009C43F84B0507F8CB97D701009387877B68
:102CF0009C433E858280797106D62AC62EC42D3724
:102D000097D701009387077A9C43BC4FADE397D7D1
:102D10000100938727799C430547F8CFA247A1CBB1
:102D200097D70100938707789C4391073E85EFD0A2
:102D30005F922247FD576310F70297D701009387F0
:102D400067769C439107BE8517E5010013058591C1
:102D5000EFD09F8519A897E70100938727929C439E
:102D60002247BA973ECE7245353CEFD02FEAE53583
:102D7000653D97D701009387E7729C43BC4F3ECCDB
:102D8000E2479DC3B24789CB97D7010093878771EC
:102D90009C4323AC070409A897D701009387877049
:102DA0009C43B84F7D17B8CF97D701009387876FA3
:102DB0009C4323AE07044535E2473E85B25045614A
:102DC0008280797106D62AC62EC432C236C0A93D89
:102DD00097D701009387076D9C43F84F8947630D90
:102DE000F70697D701009387E76B9C43B44F3247B0
:102DF0001347F7FF758FB8CF97D701009387876A7E
:102E00009C430547F8CF8247A1CB97D70100938712
:102E100067699C4391073E85EFD0BF830247FD570A
:102E20006310F70297D701009387C7679C43910708
:102E3000BE8517E501001305E582EFD0EFF619A86E
:102E400097E70100938787839C430247BA973ECC5C
:102E50006245893AEFD08FDBFD3BF933924789CB4E
:102E600097D70100938707649C43B84F924798C354
:102E700097D70100938707639C43F84F85476314F6
:102E8000F70002CE31A897D701009387A7619C4332
:102E9000B44F22471347F7FF758FB8CF85473ECE13
:102EA00097D70100938707609C4323AE07046533DF
:102EB000F2473E85B25045618280797106D62AC6B6
:102EC0002EC432C236C085473ECEB24781E773700A
:102ED000043001A0B2473ECC813B824789C7E2471C
:102EE000B84F824798C3E247FC4F3ECAE2470947C2
:102EF000F8CF1247914763EEE704924713972700F4
:102F000097D7010093878710BA97984397D7010006
:102F10009387C70FBA978287E247B84FA2475D8F62
:102F2000E247B8CF3DA0E247BC4F13871700E24706
:102F3000B8CF05A0E2472247B8CF21A8524789471A
:102F40006306F700E2472247B8CF21A002CE11A0C6
:102F5000010052478547631AF706E24791073E850D
:102F6000EFD02FEFE247D85797D7010093874771EB
:102F70009C4363F9E700E247D85797D7010093874E
:102F8000277098C3E247D857BA878A07BA978A0743
:102F900017D701001307C75A3E97E2479107BE852E
:102FA0003A85EFD06FE0E2479C5781C773700430D9
:102FB00001A0E247D85797D701009387A74E9C43BB
:102FC000DC5763F4E700EFD06FC47131F2473E8500
:102FD000B25045618280397106DE2ACE2ECC32CACB
:102FE00036C83AC685473ED6F24781E7737004304B
:102FF00001A0F2473ED4EFD04FCFAA873ED2C247BE
:1030000089C7A257B84FC24798C3A257FC4F3ED0BA
:10301000A2570947F8CF5247914763EEE704D247DA
:103020001397270097D70100938787FFBA97984394
:1030300097D701009387C7FEBA978287A257B84FE8
:10304000E2475D8FA257B8CF3DA0A257BC4F138770
:103050001700A257B8CF05A0A2576247B8CF21A842
:10306000025789476306F700A2576247B8CF21A0ED
:1030700002D611A0010002578547631DF708A25729
:103080009C5781C77370043001A097D701009387C4
:10309000E7609C43A1EBA25791073E85EFD06FDB21
:1030A000A257D85797D701009387875D9C4363F950
:1030B000E700A257D85797D701009387675C98C35A
:1030C000A257D857BA878A07BA978A0717D7010035
:1030D000130707473E97A2579107BE853A85EFD061
:1030E000AFCC11A8A257E107BE8517D50100130583
:1030F000A554EFD06FCBA257D85797D7010093872D
:10310000673A9C43DC5763F7E700B24781C7B24791
:10311000054798C392573E85EFD02FBCB2573E85E6
:10312000F25021618280797106D62AC62EC4B24738
:1031300081E77370043001A0B2473ECEEFD0EFBA02
:10314000AA873ECCF247FC4F3ECAF2470947F8CF68
:10315000F247BC4F13871700F247B8CF5247854755
:10316000631DF708F2479C5781C77370043001A0B4
:1031700097D70100938787529C43A1EBF2479107B1
:103180003E85EFD00FCDF247D85797D701009387F0
:10319000274F9C4363F9E700F247D85797D70100C0
:1031A0009387074E98C3F247D857BA878A07BA97CA
:1031B0008A0717D701001307A7383E97F2479107F0
:1031C000BE853A85EFD04FBE11A8F247E107BE8514
:1031D00017D5010013054546EFD00FBDF247D8576C
:1031E00097D701009387072C9C43DC5763F7E700D0
:1031F000A24781C7A247054798C3E2473E85EFD063
:10320000CFAD0100B25045618280797106D62AC6E1
:10321000B2473ECCE24799E797D7010093878728CA
:103220009C4311A0E2473ECC0134E247F84F894766
:103230006318F700E24723AE070485473ECE11A08E
:1032400002CE113CF2473E85B250456182800111A9
:1032500006CE02C61D2B97D70100938767479C4374
:103260009DC38148014881470947814613060040B4
:1032700097D50100938505DC170500001305051B94
:10328000EFE0AF852AC6B24781E77370043001A032
:10329000B2473E85F24005618280397106DE2ACE52
:1032A0002ECC32CA36C83AC6E24799E302D62DA8D8
:1032B0001305C002EF00302A2AD6B25795C7F12174
:1032C000B257724798C3B257624798CFB257524726
:1032D000D8CFB257424798D3B2573247D8D3B25714
:1032E00091073E85EFD04FABE24781E77370043022
:1032F00001A0B2573E85F25021618280397106DE0D
:103300002ACE2ECC32CA36C83AC602D6F24781E758
:103310007370043001A097D701009387673B9C43EB
:10332000B5CBE2473ED0D2473ED2F2473ED46247C9
:10333000954763C4E704EFF0AFF22A87894763102B
:10334000F70297D701009387A7389C43181081464E
:103350003246BA853E85EFD0AFE02AD625A897D76A
:1033600001009387E7369C43181081460146BA85D1
:103370003E85EFD0EFDE2AD631A897D7010093879C
:1033800027359C43181081464246BA853E85EFD0CA
:103390000FF32AD6B2573E85F25021618280011187
:1033A0002AC6B2473ECEB24781E77370043001A00F
:1033B000F2479C433E8505618280797106D62AC614
:1033C0002EC497D70100938727309C43DC47DC4706
:1033D0003ECEF24791073E85EFD0AFA7F247D84FD8
:1033E0008547631BF702F247984FB247BA97B24638
:1033F0002246BE857245B9222A878547631EF7009B
:1034000001478146324681457245CD3D2ACCE2478F
:1034100081E77370043001A0F247DC537245829754
:103420000100B25045618280797106D62AC63C08F7
:103430003E8541282ACEE247BE8572451920692281
:10344000FDB7797106D62AC62EC4EFE06FF93C08A5
:103450003E8545282ACEE247B9EFA24799EB32478D
:10346000F24763E8E700EFE06FF9F2453245B13724
:10347000A9A0A24781CF97D70100938727259C4316
:103480009C4393B7170093F7F70F3EC497D70100FB
:103490009387072494433247F247B307F740224605
:1034A000BE853685EFD0FFDDEFE04FF5AA8791E7C7
:1034B000EFC0DFF519A0EFE06FF40100B2504561F5
:1034C000828001112AC697D701009387E71F9C438A
:1034D0009C4393B7170093F7F70F3E87B24798C303
:1034E000B2479C4391EB97D701009387E71D9C431C
:1034F000DC479C433ECE11A002CEF2473E850561DB
:103500008280797106D62AC6EFE01F842ACE97D72B
:1035100001009387271C9C4372476377F700692A51
:10352000B247054798C321A0B24723A0070097D709
:1035300001009387271A724798C3F2473E85B2501D
:1035400045618280797106D62AC62EC432C236C041
:1035500002CEB2472247D8C3B247324798CB224760
:10356000924763E8E702124782471D8FB2479C4F9C
:103570006365F70085473ECE99A097D701009387F2
:10358000E7149843B2479107BE853A85EFD0CF85BF
:103590003DA0124782476379F7002247824763655F
:1035A000F70085473ECE21A897D701009387C71122
:1035B0009843B2479107BE853A85EFD0EF82F24734
:1035C0003E85B25045618280797106D6D9A0A24766
:1035D00063C0070CC2473ECEF247DC4B91C7F247AF
:1035E00091073E85EFD0EF865C003E85193F2ACCDF
:1035F000A2472547636FF7081397270097D7010065
:103600009387C7A3BA97984397D70100938707A3D7
:10361000BA9782873247F2479C4FBA973247BA86A9
:103620006246BE857245393F2A8785476313F70690
:10363000F247DC5372458297F247D84F8547631AA9
:10364000F7043247F2479C4FBA97014781463E86BE
:103650008145724565312ACAD24785EF73700430BF
:1036600001A03247F24798CFF2479C4F81E7737031
:10367000043001A0F247984FE247BA97E24662460B
:10368000BE857245C13531A07245EF00C07F11A0E3
:10369000010097D701009387A7039C433800814618
:1036A0000146BA853E85EFD06FD8AA87E39107F22D
:1036B0000100B25045618280797106D671A097D71A
:1036C0000100938767009C43DC479C433ECC97D71F
:1036D0000100938767FF9C43DC47DC473ECAD24723
:1036E00091073E85EFC0FFF6D247DC5352458297E3
:1036F000D247D84F85476319F704D2479C4F62479A
:10370000BA973EC84247E24763F4E702D2474247CE
:10371000D8C3D247524798CB97D701009387C7FAAF
:103720009843D2479107BE853A85EFC0FFEB29A8A1
:1037300001478146624681455245C9362AC6B2478D
:1037400081E77370043001A097D701009387C7F712
:103750009C439C43ADF797D701009387E7F69C43C2
:103760003ECE97D70100938767F6984397D701001D
:10377000938787F598C397D70100938727F57247FA
:1037800098C30100B25045618280411106C6EFF036
:10379000AFC997D701009387A7F39C43C9E717D513
:1037A00001001305E5EFEFC0FFDB17D5010013059E
:1037B00065F0EFC03FDB97D701009387E7F017D79D
:1037C00001001307E7ED98C397D70100938707F02F
:1037D00017D70100130707EE98C30146B1451145FD
:1037E000EFC07FF72A8797D70100938767EE98C3CA
:1037F00097D701009387C7ED9C4381E7737004302E
:1038000001A097D701009387A7EC9C4389CF97D756
:1038100001009387E7EB9C4397D50100938585844E
:103820003E85EFD05F9CEFF00FC30100B240410135
:103830008280797106D62AC6B2473ECEB24781E76A
:103840007370043001A0EFF02FBEF247DC4BB337AA
:10385000F00093F7F70F3ECCEFF0EFBFE2473E8565
:10386000B25045618280797106D62AC6B2473ECEF3
:10387000B24781E77370043001A0EFF0EFBAF2476E
:103880009C533ECCEFF02FBDE2473E85B2504561E0
:103890008280797106D62AC62EC4B2473ECEB24780
:1038A00081E77370043001A0EFF00FB8F2472247B0
:1038B00098D3EFF04FBA0100B250456182800111F8
:1038C00006CE714549292AC6B24789CBB24723A003
:1038D0000700B24791073E85EFC0DFC8B2473E857B
:1038E000F24005618280397106DE2AC62EC432C2DA
:1038F00036C0B2473ED402D21247B70700FFF98F55
:1039000081C77370043001A0924781E7737004305F
:1039100001A0EFF0EF94AA8799E3824799E38547E6
:1039200011A0814781E77370043001A0EFE04FAB35
:10393000A2579C433ED0A245324585240257A24758
:103940005D8F9247F98F12476310F7020257A24723
:10395000D98F3ED6A2579843924793C7F7FF7D8FE2
:10396000A25798C302C025A0824799CFA257938639
:1039700047001247B7070005D98F0246BE85368536
:10398000EFE03F8902D621A0A2579C433ED6EFE04C
:10399000EFA62ACE8247B1CBF24799E3EFC01FA72B
:1039A000EFF06FAF2AD63257B7070002F98F85EBD9
:1039B000EFF08FA7A2579C433ED632579247F98F1C
:1039C0001247631AF700A2579843924793C7F7FF2D
:1039D0007D8FA25798C3EFF00FA885473ED232578C
:1039E000B7070001FD17F98F3ED6B2573E85F2505A
:1039F000216182805D7186C62ACE2ECC32CA36C83D
:103A00003AC6F2473EDA02DC02D8F24781E7737029
:103A1000043001A06247B70700FFF98F81C77370B8
:103A2000043001A0E24781E77370043001A0EFF099
:103A30002F83AA8799E3B24799E3854711A081476D
:103A400081E77370043001A0EFE08F99D2579C4357
:103A50003ED64246E245325575242AD4A25799CF24
:103A6000B2573EDE02C6D247A9CBD2579843E247AF
:103A700093C7F7FF7D8FD25798C381A0B24781E7E4
:103A8000B2573EDE1DA8D24791C76257B707000163
:103A9000D98F3EDCC24791C76257B7070004D98F60
:103AA0003EDCD257938647006247E257D98F3246B1
:103AB000BE853685EFE0EFF502DEEFE02F942AD2E7
:103AC000B247B9CB925799E3EFC05F94EFF0AF9C48
:103AD0002ADE7257B7070002F98F8DEBEFF0CF9413
:103AE000D2579C433EDE4246E2457255212CAA87BE
:103AF00099CBD24789CBD2579843E24793C7F7FF78
:103B00007D8FD25798C3EFF00F9502D87257B70741
:103B10000001FD17F98F3EDEF2573E85B640616128
:103B20008280797106D62AC62EC4B2473ECEB247ED
:103B300081E77370043001A02247B70700FFF98FB7
:103B400081C77370043001A0EFF00F8EF2479C43E1
:103B50003ECCF2479843A24793C7F7FF7D8FF247C9
:103B600098C3EFF04F8FE2473E85B25045618280A7
:103B7000797106D62AC6B2473ECEEFC01F97AA87F4
:103B80003ECCF2479C433ECAE2473E85EFC0FF94DD
:103B9000D2473E85B250456182805D7186C62AC695
:103BA0002EC402DCB2473ED802DAB24781E7737016
:103BB000043001A02247B70700FFF98F81C7737057
:103BC000043001A0C25791073ED6B257A1073ED498
:103BD000EFE00F81B257DC473EDEC2579843A24761
:103BE0005D8FC25798C3BDA8F257DC433ED2F2574F
:103BF0009C433ED002DA0257B70700FFF98F3ECE52
:103C00000257B7070001FD17F98F3ED07247B7077B
:103C10000004F98F89EBC25798438257F98F89CFF7
:103C200085473EDA11A8C25798438257F98F025749
:103C30006314F70085473EDAD2579DC37247B70732
:103C40000001F98F89C762578257D98F3EDCC2576E
:103C50009843B7070002D98FBE857255EFE00FF980
:103C600092573EDE7257A257E310F7F8C2579843B7
:103C7000E25793C7F7FF7D8FC25798C3EFD01FF865
:103C8000C2579C433E85B64061618280797106D6F9
:103C90002AC6B2473ECEF24791073ECCEFD05FF442
:103CA0000DA0E247D847E247A1076315F7007370FC
:103CB000043001A0E247DC47B70500023E85EFE093
:103CC000EFF2E2479C43F1FF7245752AEFD01FF3F4
:103CD0000100B25045618280011106CE2AC62EC471
:103CE000A24532455D3D0100F2400561828001112F
:103CF00006CE2AC62EC4A245324525350100F24023
:103D00000561828001112AC62EC432C202CE9247BA
:103D100081EB3247A247F98F81CF85473ECE09A874
:103D20003247A247F98F22476314F70085473ECEFA
:103D3000F2473E850561828001112AC6B2473ECC1A
:103D4000B24799E302CE21A0E2479C4F3ECEF24714
:103D50003E8505618280397106DE2AC602D2EFD027
:103D60003FE897670300938727989C4381EB552290
:103D70009767030093874797054798C3B24789CF52
:103D8000A1473E87B247BA973EC6B2478D8B89C7D7
:103D9000B247F19B91073EC6B247F9CB3247E56780
:103DA000ED1763E7E70C976703009387E7923ED42C
:103DB00097670300938747929C433ED631A0B25742
:103DC0003ED4B2579C433ED6B257DC43324763F5EC
:103DD000E700B2579C43E5F7325797670300938794
:103DE00027906307F708A2579C432147BA973ED212
:103DF000B2579843A25798C3B257D843B247B307B4
:103E0000F740214706076378F7043257B247BA975D
:103E10003ECEB257D843B2471D8FF247D8C3B257F0
:103E20003247D8C3F247DC433ECC97670300938701
:103E3000A78A3ED021A082579C433ED082579C4304
:103E4000DC436247E3E9E7FE82579843F24798C3B1
:103E50008257724798C397C701009387E7659843D5
:103E6000B257DC431D8F97C701009387E76498C35F
:103E7000EFD0DFD8925799E3EF00103292573E858A
:103E8000F25021618280797106D62AC6B2473ECCB3
:103E9000B247BDC3A147B307F0406247BA973ECCD3
:103EA000E2473ECAEFD0DFD3D247DC433EC8976734
:103EB0000300938767823ECE21A0F2479C433ECE0B
:103EC000F2479C43DC434247E3E9E7FEF24798436D
:103ED000D24798C3F247524798C3D247D84397C7AF
:103EE00001009387675D9C433E9797C701009387C6
:103EF000A75C98C3EFD09FD00100B250456182808B
:103F000097C701009387475B9C433E8582800100F1
:103F10008280411197C701009387477CF19B3EC681
:103F2000975703009387477B324798C397570300FF
:103F30009387877A23A20700975703009387477ACE
:103F400065677117D8C3975703009387677923A0D4
:103F50000700B2473EC4A24765677117D8C3A2479E
:103F6000175703001307C77798C3010041018280E8
:103F700001112AC62EC432C2A2473ECEB2473ECC61
:103F80003247A247D98F8D8BA1E319A8F2479843F6
:103F9000E24798C3E24791073ECCF24791073ECEF5
:103FA0009247F5173247BA976247E361F7FE29A8AF
:103FB0007247930717003ECEE2479386170036CC30
:103FC000034707002380E70032479247BA976247CA
:103FD000E360F7FEB2473E850561828001112AC683
:103FE0002EC432C232479247D98F8D8B9DEFA247A4
:103FF00093F7F70F3ECAD247A2075247D98F3ECA5E
:10400000D247C2075247D98F3ECAB2473ECE39A0E7
:10401000F247138747003ACE524798C33247924738
:10402000BA977247E366F7FE1DA0B2473ECC11A8CF
:10403000E247138717003ACC22471377F70F238004
:10404000E70032479247BA976247E363F7FEB24709
:104050003E850561828001112AC6B2473ECE21A06D
:10406000F24785073ECEF24783C70700F5FB72474C
:10407000B247B307F7403E850561828001112AC629
:104080002EC4B247138717003AC683C70700A30F91
:10409000F100A247138717003AC483C70700230F14
:1040A000F1008347F10199C70347F1018347E1011B
:1040B000E309F7FC0347F1018347E101B307F74048
:1040C0003E850561828001112AC62EC4B2473ECECC
:1040D00001002247930717003EC4F247938617005A
:1040E00036CE034707002380E70083C70700F5F3B8
:1040F000B2473E850561828001112AC602CE02CCFC
:1041000021A0B24785073EC6B24703C70700930701
:104110000002E308F7FEB24703C707009307D00287
:104120006309F700B24703C707009307B0026311A2
:10413000F704B24783C70700938737FD93B717008B
:1041400093F7F70F3ECCB24785073EC615A07247DE
:10415000BA878A07BA9786073ECEB24713871700F9
:104160003AC683C70700938707FD7247BA973ECECA
:10417000B24783C70700E1FFE24789C7F247B307A9
:10418000F04011A0F2473E850561828001112AC6E8
:1041900097570300938707579C4393861700175739
:1041A00003001307275614C332471377F70F9756A8
:1041B000030093862659B6972380E7003247A94724
:1041C000630BF700975703009387C75398439307F0
:1041D00000046315F704975703009387A7563ECE54
:1041E00005A8F247138717003ACE03C70700B707A1
:1041F00010F0938707F098C3975703009387875071
:104200009C431387F7FF975703009387A74F98C3E3
:10421000975703009387074F9C43E1F781473E85FB
:10422000056182804D7123261114232481142322D9
:10423000911423202115232E3113232C4113232ADB
:1042400051132ACE2ECC32C836CA3AC63EC442C218
:1042500023260112B2473E8A814AC24752485286FB
:10426000D6863E85C285EF10E03FAA872E883E861F
:10427000C2868327C112138717002326E1123287D3
:104280008A07141AB69723AEE7EEB2473E848144FC
:10429000D247268763E8E702D24726876396E7007E
:1042A000C247228763E0E702B2473E8981494A86D6
:1042B000CE864245D245EF00305DAA872E883EC8A3
:1042C00042CA49BF010029A0F247E2451245829740
:1042D000A2471387F7FF3AC40327C112E346F7FE4C
:1042E00025A88327C1128A07181ABA9703A7C7EF10
:1042F0008327C1128A07141AB69783A6C7EFA5476A
:1043000063F5D7009307700519A093070003BA97C8
:104310007247E2453E8502978327C1121387F7FF54
:104320002326E112E34FF0FA01008320C114032495
:10433000811483244114032901148329C113032AFE
:104340008113832A41137161828041112AC62EC4D0
:10435000A2460547635ED700B2479C439D07E19B99
:1043600093868700324714C303A847009C4335A0B7
:10437000224719CB3247184313064700B24690C272
:104380001843BA87014811A832471843130647005B
:10439000B24690C21843BA8701483E85C2854101A2
:1043A000828041112AC62EC4A2460547635ED7000B
:1043B000B2479C439D07E19B93868700324714C315
:1043C00003A847009C4305A8224701CF3247184362
:1043D00013064700B24690C21843BA877D873A88D1
:1043E00019A83247184313064700B24690C2184333
:1043F000BA877D873A883E85C285410182803971BE
:1044000006DE22DC26DA2AC62EC432C236C011A845
:1044100063070424924785073EC2B247A24522851E
:104420008297924783C707003E8493075002E311A7
:10443000F4FE924785073EC292473EC893070002AA
:10444000A30BF100FD573ECEFD573ECC02D0924764
:10445000138717003AC283C707003E849307D4FD31
:10446000130750056364F71E1397270097C70100D1
:10447000938747C0BA97984397C70100938787BF30
:10448000BA9782879307D002A30BF100C9B79307AD
:104490000003A30BF10065BF02CC6247BA878A070D
:1044A000BA978607A297938707FD3ECC924783C7AA
:1044B00007003E849307F00263D6870293079003B8
:1044C00063C28702924785073EC2C1BF82471387F6
:1044D00047003AC09C433ECC39A0F247E3D907F6E7
:1044E00002CEB5B70100F247E3D307F6E2473ECE6E
:1044F000FD573ECCA9BF825785073ED089BF824772
:10450000138747003AC09C433247A2453E85029735
:10451000B1A28247138747003AC0844389E497C415
:1045200001009384A4B4F2476357F0040347710178
:104530009307D0026301F704E247BE852685EF00AA
:1045400070322A87F247998F3ECE11A883477101B6
:104550003247A2453E850297F247FD173ECEF2470D
:10456000E346F0FE09A8B247A2452285829785045A
:10457000F247FD173ECE83C704003E841DC0E247CC
:10458000E3C307FEE247FD173ECCE247E3DD07FC4D
:1045900009A8B247A245130500028297F247FD170A
:1045A0003ECEF247E347F0FE55A88A8782553E8506
:1045B000CD3BAA872E883ED442D6A2573258C28716
:1045C00063D90702B247A2451305D0028297A255CC
:1045D000325681470148B386B740368533B5A700C8
:1045E0003307C840B307A7403E87B6873A883ED412
:1045F00042D6A9473ED21DA8A9473ED215A0A14741
:104600003ED239A885473ED0B247A24513050003E4
:104610008297B247A245130580078297C1473ED2D1
:104620008A8782553E8515332AD42ED61257834762
:1046300071013E88F2472256B256A2453245DD3618
:1046400031A8B247A2452285829709A8B247A24560
:10465000130550028297C2473EC20100D9B3010040
:10466000F2506254D2542161828041112AC6B707A8
:1046700010F0938707F2324798C301A05D7106D608
:104680002AC62EDA32DC36DEBAC0BEC2C2C4C6C604
:104690009C0891173ECEF247BE86324681451705EB
:1046A00000001305E5AEA13B81473E85B250616134
:1046B000828001112AC62EC41EC2A2473ECEF247F6
:1046C0009C4332471377F70F2380E700F2479C4360
:1046D00013871700F24798C30100056182801D719E
:1046E00006DE2AC62EC4B2C4B6C6BAC8BECAC2CC7A
:1046F000C6CE9C103ED25C084C081706000013067C
:1047000086FB7D779346F7FF0565130505803388A3
:10471000A5003378E8001368783B23A007013295A1
:10472000698F13677733D8C333F7D50093154701E3
:1047300037870300130737394D8F98C73377D60073
:10474000931647013707030013077706558FD8C71D
:104750000F100000B2473ED69C10A1173ED422573E
:104760005C083E857C00BA862246BE854939B24740
:1047700023800700B2473E87B257B307F7403E8514
:10478000F250256182804111370510F0130545F480
:1047900008412AC6370510F0130505F408412AC45C
:1047A000370510F0130545F40841B248E39EA8FC14
:1047B00032452A8381431317030081462245AA8587
:1047C0000146B3E7B6003368C700370710F013059A
:1047D00087F48565938505FA0146B386B700B688E8
:1047E000B3B8F8003307C800B387E8003E87B68740
:1047F0003A881CC123220501010041018280411138
:1048000006C651379307000873A047300100B24035
:1048100041018280011106CE2AC617C50100130589
:10482000E59AEFF0BFE50100F240056182800111D9
:1048300006CE2AC617C501001305C599EFF01FE47F
:104840000100F24005618280797106D62AC602CE47
:1048500029A00100F24785073ECE724785679387FE
:104860007738E3D8E7FE17C5010013052597EFF069
:10487000FFE0F1BF411106C60145152A0100B24013
:1048800041018280011106CE02C6EF00E0752A8741
:104890008547630CF70017C501001305A594EFF0D9
:1048A000FFDDB24793E727003EC6B2473E85F240A0
:1048B00005618280011106CE02C66D3F1707000018
:1048C00013076704814605469305400617C5010096
:1048D00013050593EFE07F9C2AC6B24799CBEFD032
:1048E000AFC6AA87014781463E8685453245EFE03F
:1048F000FFA002C4EFD0EFA481473E85F2400561DE
:104900008280797106D62AC697C701009387C7B9F6
:104910009C431387470697C701009387E7B898C35E
:1049200097C70100938787B89C431387470697C7AB
:1049300001009387A7B798C397C701009387C7B6AD
:1049400098439307F07C63D3E70497C701009387EC
:10495000A7B59C431387078397C701009387C7B404
:1049600098C30D372ACEF24799EB97C7010093877A
:10497000E7B3984385679387F77663DBE700F247F1
:104980003E85EFF09FCEEFD0AFA321A0010011A094
:104990000100B250456182807370043001A00100B3
:1049A000828041112AC62EC47370043001A0011107
:1049B00006CE2AC6814801488147324797560300F0
:1049C000938646DC1306004097C501009385058455
:1049D000170500001305C512EFC03F90814801483C
:1049E00081473247975603009386E6D91306004065
:1049F00097C501009385058217050000130525243E
:104A0000EFC0BF8D81480148814732479756030068
:104A1000938686D71306004097C5010093850580CD
:104A20001705000013058535EFC03F8B814801480D
:104A30008147324797560300938626D513060040D8
:104A400097B501009385057E17050000130585467F
:104A5000EFC0BF888148014881473247975603001D
:104A60009386C6D21306004097B501009385057C56
:104A7000170500001305C508EFC03F8681480148AF
:104A80008147324797560300938666D0130600404D
:104A900097B501009385057A170500001305251ABF
:104AA000EFC0BF83814801488147324797560300D2
:104AB000938606CE1306004097B5010093850578CE
:104AC000170500001305852BEFC03F818148014881
:104AD00081473247975603009386A6CB13060040C2
:104AE00097B5010093850576170500001305853CF1
:104AF000EFC0AFFE0100F24005618280397106DE31
:104B000022DC2AC62317010297B701009387077496
:104B10009C433ED297B70100938787739C433ED056
:104B200097B70100938707739C433ECE9257025775
:104B3000BA853E85EF100003AA873E87F247BE85FF
:104B40003A85EF10701AAA873ECAB2473ED497B78B
:104B500001009387A76F9C433ED297B701009387CC
:104B6000276F9C433ED097B701009387A76E9C4365
:104B70003ECE92570257BA853E85EF00B07EAA8797
:104B80003E87F247BE853A85EF101016AA873ECCC5
:104B9000E2475247BA853E85EF10104CAA8793052D
:104BA00000003E85EF109007AA8763DD0702624789
:104BB000B7070080B98F5247BA853E85EF10D049BC
:104BC000AA873E87054497B701009387E7688C431F
:104BD0003A85EF10E077AA876343F00001449377AA
:104BE000F40F05A8E2475247BA853E85EF10D0463C
:104BF000AA873E87054497B701009387E7658C43F2
:104C00003A85EF10E074AA876343F000014493777C
:104C1000F40F81C785472317F1028317E10285FB53
:104C2000A25783D70700C207C183850713970701DF
:104C30004183A2572390E70019BF397106DE22DCB9
:104C40002AC62317010297B70100938727619C4367
:104C50003ED297B701009387A7609C433ED097B799
:104C60000100938727609C433ECE92570257BA8536
:104C70003E85EF106034AA873E87F247BE853A85AD
:104C8000EF109006AA873ECAB2473ED497B70100FC
:104C90009387C75C9C433ED297B701009387475CDC
:104CA0009C433ED097B701009387C75B9C433ECEA1
:104CB00092570257BA853E85EF100030AA873E878B
:104CC000F247BE853A85EF103002AA873ECCE24714
:104CD0005247BA853E85EF103038AA879305000009
:104CE0003E85EF10A073AA8763DD07026247B7070E
:104CF0000080B98F5247BA853E85EF10F035AA87FC
:104D00003E87054497B70100938707558C433A8542
:104D1000EF100064AA876343F00001449377F40F17
:104D200005A8E2475247BA853E85EF10F032AA87C0
:104D30003E87054497B70100938707528C433A8515
:104D4000EF100061AA876343F00001449377F40FEA
:104D500081C785472317F1028317E10285FBA2571C
:104D600083D70700C207C1838507139707014183D3
:104D7000A2572390E70019BF5D7186C6A2C42AC658
:104D8000A9473EDA231D0102B2473ED8D2578A070F
:104D90003E85EFE05FFC2AD6930700003ED43ED26A
:104DA0003ECE02DEB1A0F246F2578A0732573304F4
:104DB000F70097B701009387274B8C433685EF00A8
:104DC000705AAA871CC0724797B701009387C749DA
:104DD0008C433A85EF001059AA873E87A257BE85BB
:104DE0003A85EF003058AA873ED4F25785073EDE59
:104DF0007257D257E369F7FA02DE05A0F2578A0725
:104E00003257BA979C431257BA853E85EF009055AA
:104E1000AA873ED2F25785073EDE7257D257E36F1C
:104E2000F7FCA2571257BA853E85EF10F022AA87E9
:104E30003ED08257930500003E85EF10205EAA8782
:104E400063D307020257054497B7010093870742CF
:104E50008C433A85EF10805CAA8763C30700014446
:104E60009377F40F0DA00257054497B7010093877D
:104E7000A73E8C433A85EF10A04DAA876343F0000C
:104E800001449377F40F81C78547231DF1028317EF
:104E9000A103E39307F0C25783D70700C207C1837A
:104EA0008507139707014183C2572390E700EDB5AB
:104EB0005D7186C6A2C42AC6A9473EDA231D010237
:104EC000B2473ED8D2578A073E85EFE0DFE82AD6C0
:104ED000930700003ED43ED23ECE02DEB1A0F246A1
:104EE000F2578A0732573304F70097B701009387C8
:104EF00027388C433685EF10205FAA871CC0724785
:104F000097B701009387C7368C433A85EF10C05D91
:104F1000AA873E87A257BE853A85EF00B044AA878C
:104F20003ED4F25785073EDE7257D257E369F7FA4F
:104F300002DE05A0F2578A073257BA979C431257F0
:104F4000BA853E85EF001042AA873ED2F257850708
:104F50003EDE7257D257E36FF7FCA2571257BA855D
:104F60003E85EF10700FAA873ED082579305000050
:104F70003E85EF10A04AAA8763D307020257054473
:104F800097B701009387872E8C433A85EF1000492D
:104F9000AA8763C3070001449377F40F0DA002575B
:104FA000054497B701009387272B8C433A85EF1070
:104FB000203AAA876343F00001449377F40F81C736
:104FC0008547231DF1028317A103E39307F0C2571E
:104FD00083D70700C207C183850713970701418361
:104FE000C2572390E700EDB5411185473EC602C484
:104FF0008DA0174703001307E778A2478607BA97E3
:1050000083D70700139707014183974603009386D0
:105010006678A2478607B69783D707006313F70021
:1050200002C6174703001307E775A2478607BA971A
:1050300083D70700139707014183974603009386A0
:105040006675A2478607B6972390E700A2478507B3
:105050003EC422479D47E3DEE7F8B2473E85410163
:1050600082800000B305B500930705006386B70092
:1050700003C70700631607003385A7406780000059
:10508000938717006FF09FFE130101FD2322910209
:10509000232A5101232611022324810223202103E4
:1050A000232E3101232C4101232861012326710184
:1050B00023248101232291012320A101930A0500C9
:1050C00093840500639E06381304060093090500C7
:1050D00017B901001309892163F8C512B707010048
:1050E000138B05006378F6101307F00F3337C700F2
:1050F00013173700B357E6003309F9008346090058
:105100003387E60093060002B386E640638C060010
:10511000B394D40033D7EA003314D600336B97002E
:10512000B399DA00935A040193850A0013050B0022
:10513000EF1050411309050093850A00931B0401E9
:1051400013050B00EF10903B93DB0B01930405005C
:105150009305050013850B00EF1090371319090113
:1051600093D70901B367F900138A040063FEA7000F
:10517000B3878700138AF4FF63E8870063F6A7000C
:10518000138AE4FFB3878700B384A74093850A009E
:1051900013850400EF10103B1309050093850A00E6
:1051A00013850400EF1090359399090193040500CD
:1051B000930505001319090113850B0093D9090103
:1051C000EF101031B36939011386040063FCA900A4
:1051D000B30934011386F4FF63E6890063F4A90080
:1051E0001386E4FF13140A013364C400130A000099
:1051F0006F000013B707000113070001E36CF6EE20
:10520000130780016FF01FEF138A0600631A060070
:105210009305000013051000EF10502E1304050035
:10522000B7070100637EF4129307F00F63F4870061
:10523000130A8000B35744013309F90003470900FA
:105240009306000233074701B386E64063940612D3
:10525000B3848440130A1000135B040193050B0010
:1052600013850400EF10102E1309050093050B00A1
:1052700013850400931B0401EF10502893DB0B01EE
:10528000930405009305050013850B00EF105024CF
:105290001319090193D70901B367F900938A040030
:1052A00063FEA700B3878700938AF4FF63E8870053
:1052B00063F6A700938AE4FFB3878700B384A7400F
:1052C00093050B0013850400EF10D0271309050088
:1052D00093050B0013850400EF10502293990901E8
:1052E00093040500930505001319090113850B00AC
:1052F00093D90901EF10D01DB36939011386040059
:1053000063FCA900B30934011386F4FF63E6890046
:1053100063F4A9001386E4FF13940A013364C40004
:105320001305040093050A008320C10203248102AF
:1053300083244102032901028329C101032A810137
:10534000832A4101032B0101832BC100032C81001F
:10535000832C4100032D010013010103678000002D
:10536000B7070001130A0001E366F4EC130A800199
:105370006FF05FEC3314D40033DAE400B399DA0051
:1053800033D7EA00935A0401B394D40093850A00FA
:1053900013050A00336B9700EF10D01A13090500AC
:1053A00093850A0013050A00931B0401EF101015E2
:1053B00093DB0B01930405009305050013850B0097
:1053C000EF1010111319090113570B013367E9008E
:1053D000138A0400637EA70033078700138AF4FF53
:1053E000636887006376A700138AE4FF33078700AA
:1053F000B304A74093850A0013850400EF109014AE
:105400001309050093850A0013850400EF10100F9F
:10541000930405009305050013850B00EF10500B56
:1054200013170B011357070113190901B367E9009B
:105430001387040063FEA700B38787001387F4FF78
:1054400063E8870063F6A7001387E4FFB38787004C
:10545000131A0A01B384A740336AEA006FF0DFDF52
:1054600063ECD51EB707010063F4F6041307F00FD1
:10547000B335D7009395350033D7B60097B7010001
:105480009387C7E6B387E70003C70700130A000244
:105490003307B700330AEA4063160A021304100008
:1054A000E3E096E833B6CA00134416006FF05FE7F6
:1054B000B707000193050001E3E0F6FC93058001C6
:1054C0006FF09FFBB35CE600B3964601B3ECDC00E3
:1054D00033D4E40093DB0C01B397440133D7EA00E3
:1054E00093850B0013050400336BF700B3194601D5
:1054F000EF1050051309050093850B0013050400F8
:10550000139C0C01EF10807F135C0C0193040500C9
:105510009305050013050C00EF10807B131909019A
:1055200013570B013367E90013840400637EA7005F
:10553000330797011384F4FF636897016376A7002C
:105540001384E4FF33079701B304A74093850B004E
:1055500013850400EF10007F1309050093850B00ED
:1055600013850400EF10807993040500930505006E
:1055700013050C00EF10C07593170B0113190901E7
:1055800093D70701B367F9001386040063FEA700F1
:10559000B38797011386F4FF63E8970163F6A700CA
:1055A0001386E4FFB387970113140401B70B0100BE
:1055B0003364C4001389FBFF337D240133F92901CF
:1055C000B384A7409305090013050D00EF10407048
:1055D000935C040193050900130B050013850C006F
:1055E000EF10006F93D90901130C05009385090092
:1055F00013850C00EF10C06D130905009385090099
:1056000013050D00EF10C06C3305850193570B0196
:105610003385A70063748501330979019357050128
:10562000B387270163E6F402E392F4BCB7070100F5
:105630009387F7FF3375F50013150501337BFB00E6
:1056400033964A0133056501130A0000E37AA6CCBC
:105650001304F4FF6FF09FB9130A00001304000055
:105660006FF01FCC130101FB23248104232291043A
:10567000232E310323229103232611042320210505
:10568000232C4103232A510323286103232671037A
:10569000232481032320A103232EB101930C0500B1
:1056A000938905001304050093840500639E062674
:1056B00013090600138A060097BA0100938A0AC3E9
:1056C00063F4C514B70701006376F6129307F00F71
:1056D00063F4C700130A8000B3574601B38AFA0087
:1056E00003C70A001305000233074701330AE540E8
:1056F000630C0A00B395490133D7EC003319460116
:10570000B364B70033944C01935A090193850A009E
:1057100013850400EF1000639309050093850A00C8
:10572000131B090113850400EF10405D135B0B018F
:105730009305050013050B00EF108059939909019B
:1057400093570401B3E7F90063FAA700B387270171
:1057500063E6270163F4A700B3872701B384A7405A
:1057600093850A0013850400EF10C05D93090500BE
:1057700093850A0013850400EF10405813140401A8
:10578000930505009399090113050B0013540401B7
:10579000EF10005433E48900637AA4003304240139
:1057A000636624016374A400330424013304A44019
:1057B00033554401930500008320C1040324810470
:1057C00083244104032901048329C103032A81039B
:1057D000832A4103032B0103832BC102032C810283
:1057E000832C4102032D0102832DC1011301010508
:1057F00067800000B7070001130A0001E36EF6ECB2
:10580000130A80016FF05FED631A06009305000034
:1058100013051000EF10804E13090500B7070100B3
:10582000637AF90E9307F00F63F42701130A8000DF
:10583000B3574901B38AFA0003C70A0013050002EF
:10584000B384294133074701330AE540E30E0AEAEE
:1058500033194901B3DAE900B395490133D7EC00B4
:1058600093540901336BB70013850A009385040034
:10587000EF10404D9309050093850400931B090127
:1058800013850A00EF10804793DB0B019305050099
:1058900013850B00EF10C0439399090193570B0137
:1058A000B3E7F90033944C0163FAA700B3872701EB
:1058B00063E6270163F4A700B3872701B38AA740F3
:1058C0009385040013850A00EF10C0479309050073
:1058D0009385040013850A00EF10404293050500EC
:1058E00013850B00EF10C03E93150B01939909012E
:1058F00093D50501B3E5B90063FAA500B385250189
:1059000063E6250163F4A500B3852501B384A540B2
:105910006FF09FDFB7070001130A0001E36AF9F097
:10592000130A80016FF0DFF0E3E8D5E8B707010064
:1059300063FCF604930BF00F33B5DB001315350051
:1059400033D7A60097B701009387479AB387E7003C
:1059500083CB070093050002B38BAB00338B7541FB
:10596000631E0B0263E4360163EACC003384CC404F
:10597000B386D94033B58C00B384A6401305040028
:10598000938504006FF05FE3B70700011305000182
:10599000E3E8F6FA130580016FF09FFAB39666010B
:1059A000335D7601336DDD0033D47901B395690140
:1059B00033DC7C0193540D01336CBC0013050400EF
:1059C00093850400B31A6601EF10C037130A05006F
:1059D000938504001305040033996C01931C0D0199
:1059E000EF10C03193DC0C01130405009305050092
:1059F00013850C00EF10C02D131A0A0113570C0168
:105A00003367EA00130A0400637EA7003307A70187
:105A1000130AF4FF6368A7016376A700130AE4FF83
:105A20003307A701B309A740938504001385090034
:105A3000EF1040319385040013040500138509001D
:105A4000EF10C02B930505009304050013850C008F
:105A5000EF10002893150C011314040193D50501D0
:105A6000B365B4001387040063FEA500B385A501E8
:105A70001387F4FF63E8A50163F6A5001387E4FF2D
:105A8000B385A501131A0A01B70C0100336AEA00B5
:105A90001384FCFFB3778A0033F48A00B384A540F3
:105AA00013850700930504002326F100135A0A0109
:105AB000EF100022930905009305040013050A0066
:105AC000EF10002113DC0A01930D050093050C0073
:105AD00013050A00EF10C01F8327C100130A050039
:105AE00093050C0013850700EF10801E3305B501E8
:105AF00013D709013307A7006374B701330A9A016A
:105B0000B70701009387F7FF935507013377F70035
:105B100013170701B3F7F900B3854501B307F70081
:105B200063E6B400639EB400637CF900338657419A
:105B3000B3B7C700B385A541B385F5409307060009
:105B4000B307F9403339F900B385B440B385254133
:105B500033947501B3D767013365F400B3D565019C
:105B60006FF09FC5B7078000130101FF9387F7FF10
:105B700033F7A7002324810023202101135475014A
:105B80001359F50113D57501B3F7B7001374F40F6A
:105B90001375F50F232611002322910093D5F501EB
:105BA00013163700939737003307A440631EB918C4
:105BB0006358E00A63180506639C07009307F00F1B
:105BC000630CF40493070600130504006F00C00B78
:105BD0001307F7FF631E0702B387C700130504000E
:105BE000139757006352070A130515001307F00FA8
:105BF0006304E5323707007E93F617001307F7FFBB
:105C000093D71700B3F7E700B3E7D7006F00C007DB
:105C10009306F00F6310D402930706001305F00FEC
:105C20006F0080069306F00FE308D4FEB706000469
:105C3000B3E7D7009306B00163D6E60093071000E0
:105C40006FF09FF993060002B386E640B3D5E700F4
:105C5000B397D700B337F000B3E7F5006FF0DFF785
:105C60006304070863100404630006029306F0FF50
:105C70006316D700B387C7006FF09FF69306F00F47
:105C80001347F7FF631AD50213F777006308072855
:105C900013F7F700930640006302D7289387470065
:105CA0006F00C0279306F00FE300D5FEB70600048F
:105CB0003307E0403366D6009306B00163D6E600B2
:105CC000130710006F00C00193060002B355E600F1
:105CD0003387E6403317E6003337E00033E7E5006B
:105CE000B387E7006FF0DFEF130514009376F50F2D
:105CF000130710006340D704631804021305000063
:105D0000E30406F863860720B387C700139757009C
:105D1000E35C07F6370700FC1307F7FFB3F7E7006C
:105D2000130510006FF05FF6E30A06EE63940716A2
:105D30006FF09FEE1307F00F6300E51E3307F600C8
:105D4000935717006FF05FF46350E0086316050483
:105D5000E38607E61307F7FF63140702B307F6406D
:105D60001305040013975700E35007F2B70400042B
:105D70009384F4FFB3F49700130405006F00C0137D
:105D80009306F00FE30AD4E89306B00163D0E6026D
:105D9000930710006FF09FFC9306F00FE30ED4E61C
:105DA000B7060004B3E7D7006FF01FFE93060002AA
:105DB000B3D5E7003387E640B397E700B337F00089
:105DC000B3E7F5006FF09FF9630E0706631E040248
:105DD00013890500E30A06EA9306F0FF6318D7006B
:105DE000B387C740138905006FF0DFF79306F00F04
:105DF0001347F7FFE30AD5E89306B00163D4E60240
:105E0000130710006F0080039306F00F138905003D
:105E1000E30CD5E6B70600043307E0403366D6004E
:105E20006FF09FFD930600023358E6003387E6408B
:105E30003317E6003337E0003367E800B387E74005
:105E40006FF05FFA130714001377F70F9306100033
:105E500063CAE604631C040263180600639E07120B
:105E6000130500006F008003638C07123307F640B0
:105E700093165700B387C74063C006129307070005
:105E800063160706930700006FF09FFDE31006EA14
:105E9000639C0710B70700021305F00F13090000F9
:105EA0006F00C007B304F64013975400635407040F
:105EB000B384C7401389050013850400EF00D06E3A
:105EC0001305B5FFB394A400634A850233058540EA
:105ED0001305150013040002B3D7A4003305A44032
:105EE000B394A400B3349000B3E797001305000007
:105EF0006FF09FD9E38804F86FF01FFCB70700FC30
:105F00009387F7FF3305A440B3F7F4006FF0DFD7B2
:105F1000930706006FF05FD79307000013975700B1
:105F2000635E0700130515001307F00F6302E50811
:105F3000370700FC1307F7FFB3F7E7001307F00F6D
:105F400093D737006318E50063860700B707400062
:105F500013090000370780001307F7FF1375F50FCB
:105F6000B3F7E70013177501370580808320C10060
:105F7000032481001305F5FF33F5A7001319F90178
:105F80003365E500336525018324410003290100C1
:105F90001301010167800000138905006FF01FF5F0
:105FA000930706006FF09FF4138905006FF01FC779
:105FB000930700006FF09FF8130101FD2322910267
:105FC000232A510193547501B70A8000232021032D
:105FD00023286101938AFAFF2326110223248102D8
:105FE000232E3101232C4101232671012324810119
:105FF00093F4F40F138B0500B3FAAA001359F501BB
:10600000638804089307F00F6384F40A939A3A00B4
:10601000B7070004B3EAFA00938414F8930B000066
:1060200013557B01370480001304F4FF1375F50F3B
:1060300033746401135BFB01630C05089307F00FD5
:106040006308F50A13143400B70700043364F4003E
:10605000130515F89307000013972B003367F7001B
:106060001307F7FF9306E000B3496901338AA440A0
:1060700063E0E60A97A601009386C61F1317270060
:106080003307D700032707003307D700670007004F
:10609000638A0A0213850A00EF0010519307B5FFC7
:1060A0009304A0F8B39AFA00B384A4406FF01FF7EA
:1060B0009304F00F930B2000E3840AF6930B300057
:1060C0006FF01FF693040000930B10006FF05FF564
:1060D000630A040213050400EF00104D9307B5FF97
:1060E0003314F4009307A0F83385A7406FF09FF6B0
:1060F0001305F00F93072000E30004F69307300028
:106100006FF09FF513050000930710006FF0DFF4A8
:10611000131B540063F68A12130AFAFF13090000D6
:10612000935B0B013704010093850B001304F4FF0C
:1061300013850A00EF00903C33748B009305050033
:10614000130C050013050400EF00903893040500BC
:1061500093850B0013850A00EF00D03E1359090107
:10616000131505013365A90013090C00637E950022
:10617000330565011309FCFF6368650163769500CB
:106180001309ECFF33056501B304954093850B00BB
:1061900013850400EF00903693050500130C0500ED
:1061A00013050400EF00D032930A050093850B001D
:1061B00013850400EF0010391315050113040C00BA
:1061C000637E5501330565011304FCFF63686501B7
:1061D000637655011304ECFF3305650113190901BA
:1061E00033055541336989003335A0003364A90074
:1061F0001307FA076350E00A93777400638A070075
:106200009377F400930640006384D700130444009E
:106210009317440063DA0700B70700F89387F7FF86
:106220003374F40013070A089307E00F1354340083
:1062300063D2E70C130400001307F00F6F00800B0C
:106240001399FA0193DA1A006FF09FED9309090090
:1062500013840A0093870B0013072000E38CE7FCEC
:10626000130730006382E70813071000E392E7F892
:1062700013040000130700006F00C00793090B0010
:106280006FF09FFD37044000930900009307300032
:106290006FF09FFC93071000B387E7401307B0012E
:1062A000E348F7FC1305EA09B357F4003314A400DC
:1062B0003334800033E4870093777400638A0700E7
:1062C0009377F400130740006384E700130444004D
:1062D0009317540013543400E3DE07F8130400004E
:1062E000130710006F000001370440001307F00F80
:1062F00093090000370580001305F5FF3374A400EF
:10630000370580801305F5FF1377F70F3374A4006A
:10631000131777011395F9013364E4003365A40082
:106320008320C10203248102832441020329010244
:106330008329C101032A8101832A4101032B010121
:10634000832BC100032C810013010103678000002F
:10635000370780001307F7FF935675013378A700BE
:1063600013D675019357F50193F6F60F1305F00F49
:106370003377B7001376F60F93D5F5016398A6002F
:106380001305E0FF630E0806678000006318A6008F
:106390001305E0FF630E070667800000639406069E
:1063A000133518006314060063060704631C050018
:1063B0006394B700635ED600130510006396070070
:1063C00067800000E39E05FE1305F0FF6780000074
:1063D00063DAC6001305F0FFE38407FE130510001F
:1063E00067800000E36A07FD13050000E364E8FE30
:1063F0006FF01FFD13050000E30408FC6FF0DFFBE6
:10640000E308D6F8E31606FAE30807FA6FF05FFA36
:1064100013351800E38C06F86FF09FF937078000FA
:106420001307F7FF935675013378A70013D675014C
:106430009357F50193F6F60F1305F00F3377B70076
:106440001376F60F93D5F5016398A6001305200087
:10645000630E0806678000006318A600130520007D
:10646000630E070667800000639406061335180064
:106470006314060063060704631C05006394B700F9
:10648000635ED60013051000639607006780000066
:10649000E39E05FE1305F0FF6780000063DAC60087
:1064A0001305F0FFE38407FE13051000678000006A
:1064B000E36A07FD13050000E364E8FE6FF01FFDCB
:1064C00013050000E30408FC6FF0DFFBE308D6F8D7
:1064D000E31606FAE30807FA6FF05FFA13351800BF
:1064E000E38C06F86FF09FF9130101FD232291025E
:1064F00023202103B704800013597501232E310195
:10650000232671019384F4FF2326110223248102A0
:10651000232C4101232A51012328610123248101D5
:10652000232291011379F90F938B0500B3F4A40092
:106530009359F501630A09089307F00F6306F90AF6
:1065400093943400B7070004B3E4F400130919F876
:10655000130B000013D57B01370480001304F4FFF4
:106560001375F50F3374740193DBFB01630E05089B
:106570009307F00F630AF50A13143400B7070004F9
:106580003364F400130515F89306000093172B00ED
:10659000B3E7D7003309A9009387F7FF1307E0009B
:1065A00033CA7901930A19006360F70A17A701003B
:1065B000130707D093972700B387E70083A7070047
:1065C000B387E70067800700638A0402138504002D
:1065D000EF00807D9307B5FF1309A0F8B394F40092
:1065E0003309A9406FF0DFF61309F00F130B2000F9
:1065F000E38204F6130B30006FF0DFF5130900009F
:10660000130B10006FF01FF5630A0402130504005A
:10661000EF0080799307B5FF3314F4009307A0F8D7
:106620003385A7406FF05FF61305F00F9306200047
:10663000E30E04F4930630006FF05FF513050000DD
:10664000930610006FF09FF4370C0100130BFCFF52
:1066500093DB0401935C0401B3F4640133746401BB
:106660009305040013850400EF0080669305040081
:106670009309050013850B00EF00806513040500E6
:1066800093850C0013850B00EF008064930B0500CD
:106690009385040013850C00EF00806333058500AB
:1066A00093D709013385A70063748500B38B8B01F1
:1066B000B377650193970701B3F96901B387370190
:1066C000139467003334800093D7A7011355050155
:1066D000B367F40033047501131464003364F400E9
:1066E0009317440063D6070E9357140013741400D5
:1066F00033E487001387FA076350E00E9377740042
:10670000638A07009377F400930640006384D70000
:10671000130444009317440063DA0700B70700F836
:106720009387F7FF3374F40013870A089307E00F89
:1067300063C4E710935734006F000003138A090005
:106740001384040093060B00930720006386F60E63
:1067500093073000638AF60C1306100093070000BD
:1067600013070000E398C6F8370480001304F4FF11
:1067700037058080B3F787001305F5FF8320C1023A
:10678000032481021377F70FB3F7A70013177701DC
:106790001315FA01B3E7E70083244102032901023C
:1067A0008329C101032A8101832A4101032B0101AD
:1067B000832BC100032C8100832C410033E5A7000B
:1067C0001301010367800000138A0B006FF0DFF7ED
:1067D000930A09006FF01FF293071000B387E74098
:1067E0001307B0016340F706938AEA09B357F40030
:1067F000331454013334800033E4870093777400FA
:10680000638A07009377F400130740006384E7006E
:10681000130444009317540063CA070293573400CB
:10682000130700006FF05FF4B70740001307F00F85
:10683000130A00006FF05FF3930700001307F00FD7
:106840006FF09FF2930700006FF09FFD9307000029
:10685000130710006FF05FF1B70780009387F7FF11
:10686000130101FF33F7A7009356750113D6750185
:10687000B3F7B700232291002320210193F6F60FEE
:10688000131837001376F60F2326110023248100F6
:106890001307F00F9354F501138906001305060042
:1068A00093D5F501939737006314E60063940700CE
:1068B00093C515003387C640639A951A6356E00A5C
:1068C00063160606639C07009307F00F638CF604BB
:1068D00093070800138506006F00C0141307F7FF25
:1068E000631E0702B387070113850600139757003D
:1068F000635A0712130515001307F00F630EE532F4
:106900003707007E93F617001307F7FF93D717009A
:10691000B3F7E700B3E7D7006F00C0101306F00F1E
:10692000639EC600930708006F0040071306F00F30
:10693000E38AC6FE37060004B3E7C7001306B001BA
:106940006356E600930710006FF0DFF913060002AC
:106950003306E640B3D5E700B397C700B337F0007E
:10696000B3E7F5006FF01FF863000708639C0602A9
:10697000631808001307F00F6316E60A6F000002A1
:106980009306F0FF6316D700B38707016FF01FF679
:106990009306F00F1347F7FF6310D6021305F00FAD
:1069A0006F0040089306F00FE30AD6FEB706000416
:1069B0003307E0403368D8009306B00163D6E600A1
:1069C000130710006F00C001930600023356E80061
:1069D0003387E6403317E8003337E0003367E600DB
:1069E000B387E7006FF09FF0138516001376F50F5D
:1069F000130710006342C7066394060413050000E2
:106A00006302080263860722B387070113975700C2
:106A1000635A0700370700FC1307F7FFB3F7E700D7
:106A20001305100013F77700630A072013F7F70028
:106A3000930640006304D720938747006F0000202F
:106A4000E30E08F4E38007EEB70700021305F00F2A
:106A5000930400006F00801E1307F00F630EE51C07
:106A60003307F800935717006FF0DFFB6350E0081F
:106A700063160604E38A07E41307F7FF63140702AB
:106A8000B307F8401385060013975700E35C07F837
:106A9000370400041304F4FF33F4870013090500DE
:106AA0006F0080131306F00FE38EC6E61306B001E5
:106AB0006350E602930710006FF09FFC1306F00F7F
:106AC000E382C6E637060004B3E7C7006FF01FFE97
:106AD00013060002B3D5E7003307E640B397E7009B
:106AE000B337F000B3E7F5006FF09FF963020708D2
:106AF000639E0602631808001307F00F93840500D5
:106B00006FF09FE79306F0FF6318D700B387074144
:106B1000938405006FF05FF79306F00F1347F7FFBC
:106B20006310D602938405006FF05FE79306F00FC1
:106B3000E30AD6FEB70600043307E0403368D80006
:106B40009306B00163D6E600130710006F00C00182
:106B5000930600023356E8003387E6403317E80017
:106B60003337E0003367E600B387E7406FF05FFA42
:106B7000138716001377F70F130610006344E6041B
:106B8000639C06026318080063980712130500004F
:106B90006FF01FEC638607123307F8409316570017
:106BA000B387074163CA06109307070063100706FF
:106BB000930700006FF09FFDE31608E8E39407F6E3
:106BC0006FF09FE83304F840131754006354070430
:106BD000338407419384050013050400EF00C01CB3
:106BE0001305B5FF3314A400634A2503330525417B
:106BF0001305150013070002B357A4003305A7407F
:106C00003314A40033348000B3E787001305000079
:106C10006FF05FE1E30E04F86FF01FFCB70700FCB4
:106C20009387F7FF3305A940B377F4006FF09FDF38
:106C3000930708006FF01FDF9307000013975700BA
:106C4000635E0700130515001307F00F630EE506DA
:106C5000370700FC1307F7FFB3F7E7001307F00F40
:106C600093D737006318E50063860700B707400035
:106C700093040000370780001307F7FF1375F50F23
:106C8000B3F7E70013177501370580808320C10033
:106C9000032481001305F5FF33F5A7009394F40155
:106CA0003365E50033659500032901008324410025
:106CB0001301010167800000938405006FF01FF548
:106CC000930708006FF09FF4930700006FF01FF91F
:106CD000130605001305000093F6150063840600F3
:106CE0003305C50093D5150013161600E39605FE6F
:106CF000678000006340050663C60506138605002D
:106D0000930505001305F0FF630C060293061000BF
:106D1000637AB6006358C0001316160093961600E7
:106D2000E36AB6FE1305000063E6C500B385C540FF
:106D30003365D50093D6160013561600E39606FE6B
:106D40006780000093820000EFF05FFB1385050071
:106D5000678002003305A04063D80500B305B0404A
:106D60006FF0DFF9B305B04093820000EFF01FF938
:106D70003305A040678002009382000063CA0500CB
:106D8000634C0500EFF09FF7138505006780020054
:106D9000B305B040E35805FE3305A040EFF01FF601
:106DA0003305B04067800200B7070100637AF5023F
:106DB0009307F00FB3B7A7009397370013070002AC
:106DC0003307F740B357F500179501001305055237
:106DD000B307F50003C507003305A740678000002F
:106DE0003707000193070001E36AE5FC9307800180
:046DF0006FF0DFFC65
:02000004800278
:1000000049444C4500000000482FFEFF102FFEFF22
:100010001E2FFEFF2C2FFEFF342FFEFF5830FEFF59
:100020002030FEFF2E30FEFF3C30FEFF4430FEFF4E
:10003000546D722053766300DC35FEFFDC35FEFF25
:10004000DC35FEFF5A36FEFF2A36FEFF5036FEFF35
:10005000DC35FEFFDC35FEFF5A36FEFF2A36FEFF9A
:10006000546D725100000000286E756C6C29000000
:10007000DE43FEFFDC45FEFFD245FEFFDC45FEFF12
:10008000DC45FEFFDC45FEFFDC45FEFF5C44FEFF79
:10009000DC45FEFFDC45FEFF1444FEFF6A44FEFF24
:1000A000DC45FEFF1E44FEFF2844FEFF2844FEFF01
:1000B0002844FEFF2844FEFF2844FEFF2844FEFF9C
:1000C0002844FEFF2844FEFF2844FEFFDC45FEFFD7
:1000D000DC45FEFFDC45FEFFDC45FEFFDC45FEFFA8
:1000E000DC45FEFFDC45FEFFDC45FEFFDC45FEFF98
:1000F000DC45FEFFDC45FEFFDC45FEFFDC45FEFF88
:10010000DC45FEFFDC45FEFFDC45FEFFDC45FEFF77
:10011000DC45FEFFDC45FEFFDC45FEFFDC45FEFF67
:10012000DC45FEFFDC45FEFFDC45FEFFDC45FEFF57
:10013000DC45FEFFDC45FEFFDC45FEFFDC45FEFF47
:10014000DC45FEFFDC45FEFFDC45FEFFDC45FEFF37
:10015000DC45FEFFDC45FEFFDC45FEFFDC45FEFF27
:10016000DC45FEFFDC45FEFFDC45FEFFDC45FEFF17
:100170008E44FEFF3A45FEFFDC45FEFFDC45FEFFF8
:10018000DC45FEFFDC45FEFFDC45FEFFDC45FEFFF7
:10019000DC45FEFF8644FEFFDC45FEFFDC45FEFF3E
:1001A0008E45FEFF9445FEFFDC45FEFFDC45FEFF6D
:1001B000A244FEFFDC45FEFF8845FEFFDC45FEFF56
:1001C000DC45FEFFAC45FEFF6D69616F750A0000FE
:1001D0006D69616F75320A0068756E6772790A0021
:1001E0004572726F7220696E2073705F666C6F70FB
:1001F00073207461736B73200D0A0000436865639C
:100200006B54696D657200004D61746831000000C7
:100210004D617468320000004D6174683300000065
:100220004D617468340000004D6174683500000051
:100230004D617468360000004D617468370000003D
:100240004D61746838000000D5E9F642DD9A124528
:10025000358E65C46F12833AA4B0C2C366E4FD460E
:10026000A30100C00000B0406F1283BACFF7414134
:10027000C45FFEFF0060FEFF0C60FEFF0060FEFF3B
:100280007860FEFF0060FEFF0C60FEFFC45FFEFFB3
:10029000C45FFEFF7860FEFF0C60FEFFDC5FFEFFC8
:1002A000DC5FFEFFDC5FFEFF1460FEFF9C64FEFF70
:1002B0009C64FEFF1C65FEFF9464FEFF9464FEFFD9
:1002C0007C65FEFF1C65FEFF9464FEFF7C65FEFFFF
:1002D0009464FEFF1C65FEFF9064FEFF9064FEFFC9
:1002E0009064FEFF7C65FEFF00010202030303032E
:1002F00004040404040404040505050505050505B6
:100300000505050505050505060606060606060695
:10031000060606060606060606060606060606067D
:100320000606060606060606070707070707070765
:10033000070707070707070707070707070707074D
:10034000070707070707070707070707070707073D
:10035000070707070707070707070707070707072D
:100360000707070707070707080808080808080815
:1003700008080808080808080808080808080808FD
:1003800008080808080808080808080808080808ED
:1003900008080808080808080808080808080808DD
:1003A00008080808080808080808080808080808CD
:1003B00008080808080808080808080808080808BD
:1003C00008080808080808080808080808080808AD
:1003D000080808080808080808080808080808089D
:0803E0000808080808080808D5
:1003E8001000000000000000017A5200017C0101A9
:1003F8001B0D02004C00000018000000844CFEFF9A
:10040800DC05000000440E307089039507810188DF
:100418000292049305940696089709980A990B9AEC
:100428000C0370020AC144C844C944D244D344D41A
:1004380044D544D644D744D844D944DA440E004479
:100448000B00000050000000680000001052FEFF82
:100458000005000000440E50748802890393059932
:100468000B810192049406950796089709980A9AB1
:100478000C9B0D0320010AC144C844C944D244D38B
:1004880044D444D544D644D744D844D944DA44DB88
:08049800440E00440B000000BB
:1004AC00AAAAAAAA08000000FC8F010009000000FB
:040000058000004037
:00000001FF
